:100000000C948C040C94B4040C94B4040C94B404B8
:100010000C94B4040C94B4040C94B4040C94B40480
:100020000C94B4040C94B4040C94281F0C94A81FD2
:100030000C94B4040C94B4040C94B4040C94B40460
:100040000C94B4040C94B4040C94B4040C94B40450
:100050000C94B4040C94B4040C94B4040C94C63002
:100060000C94B4040C94B4040C94B4040C94B40430
:100070000C94B4040C94B4040C94B4040C94B40420
:100080000C94B4040C94B4040C94B4040C94B40410
:100090000C94B4040C94B4040C94B4040C94B40400
:1000A0000C94B4040C94B4040C94B4040606000C30
:1000B0000C1E1E3F1E3F0C1E000C0606000C0C1EE4
:1000C000123F123F0C1E000C20204F4B20200044FA
:1000D000656661756C740042617564207261746557
:1000E0003A0057656C636F6D6520746F20746865A6
:1000F0002041726475626F79206465736B746F70F0
:1001000020656E7669726F6E6D656E74210A577226
:10011000697474656E206279204A616D6573204848
:100120006F7761726420666F722074686520417217
:100130006475626F792067616D65206A616D203436
:1001400020776865726520746865207468656D65E0
:100150002077617320276E6F7420612067616D6561
:10016000272E0A5468652067726170686963616C44
:10017000207374796C6520697320626173656420F3
:100180006F6E2074686520636C6173736963204DC2
:100190006163696E746F736820696E7465726661FD
:1001A00063652E0037383941420A34353643440AF4
:1001B00031323345460A3000566F6C746167653AD8
:1001C000200054656D70657261747572653A200027
:1001D000416C6C206F6E004F666600426C75650066
:1001E000477265656E0052656400456E61626C65BC
:1001F0002072656D6F74652067616D657061640064
:100200004D6F75736520737065656400456E61623E
:100210006C652072656D6F7465206D6F7573650018
:10022000456E61626C652072656D6F7465206B65EB
:1002300079626F61726400486F6C6420412B4220C8
:10024000746F2063616E63656C0052656D6F7465D9
:100250002067616D6570616420656E61626C6564C4
:10026000005072657373204120746F2063616E6368
:10027000656C0052656D6F7465206D6F75736520D8
:10028000656E61626C65640052656D6F7465206BAC
:100290006579626F61726420656E61626C6564008D
:1002A000D5F08D14A1C881CFD9F1AF2000090B0082
:1002B000020004007070F8F0FB70F8007000040099
:1002C0000200000000000000070207000700000015
:1002D000000000050B000000FE1EFF00FE000000F5
:1002E000030007000700070003070B00FCFCFE5C8F
:1002F000FFACFFFCFFFCFE00FC0003030703070349
:1003000007030703070003090B00FE54FE54FF0018
:10031000FF00FF00FF54FF54FE00FE000301030135
:1003200007000700070007010701030003090B008E
:10033000FFAAFFFEFFFEFF00FF7AFF00FFFEFF00A7
:10034000FF0007020703070307030702070307036A
:10035000070007050B00FE24FF50FF24FF00FE00EE
:10036000030107000701070003070B007800FF06E1
:10037000FF06FF06FF00FF007800000000000000FD
:1003800007000000000000090B00FFFEFFAAFFAA03
:10039000FFA0FFAEFFACFEE8FC00F8000703070279
:1003A00007020702070207020703070007070345C2
:1003B0004550524F4D000000630900000008803690
:1003C000E9024261747465727900009E06000000C3
:1003D000085536D302546865726D616C00001308CD
:1003E000000000085536AD024C45440000000000F6
:1003F00000B6040000080A4A3400000000000000B3
:1004000000000000000000000000000069035465C7
:10041000726D696E616C00B80D0000000880365383
:100420000352656D6F7465000000820500000E08C0
:1004300064362D034E6F74657300000000570BB8CF
:100440000204096036000000000000000000000007
:100450000000000000000000090900FEFAFFFAFF9A
:10046000F8FEF8FCF8FCF8FCF8FC00FC00010001C8
:100470000001000100010001000100010001580419
:10048000417070730000000000A1100C040810609F
:10049000225804537973000000000000A110AD033E
:1004A000200840368703526561646D65000000577F
:1004B0000B0000040960360000000000000000008E
:1004C00000000000000000000000F90441726475A3
:1004D000626F790000A1107E0400086022417264FE
:1004E00075626F790057656C636F6D6520746F205E
:1004F00041726475626F792E00090B00FFFEFF6286
:10050000FF22FF62FFE2FF62FFFEFF00FF00070322
:100510000703070207030703070307030700070092
:10052000004908B400BEF67B7AA59455B848002966
:1005300044442A15A00B420050030200082590767F
:10054000BA595CC59EC53892E6F33A73BAE590771E
:10055000BA773A084008502A441CE08852E5085609
:100560008E77B677B8728CD6BA739E739272AEB726
:10057000B6E95C64AAB7B4929CBEB6D6B656AAD702
:100580009276EE77B47138E948B6AEB6AAB6F6B54B
:10059000B4B548E59C694C9124642E5400001C4479
:1005A000000EAE9ABA0E8C2EAE0ECE56D0553B93A0
:1005B000B44144415197B4494417B61AB60AAAD671
:1005C000D3766717900F389A8C16AE16BA16F615B2
:1005D000B4B52B1C5E6B4C4948C95A540056E246D0
:1005E000696C65000000000000000000004C6F61B5
:1005F0006400000000000000000800536176650000
:1006000000000000000000010044756D70204545A9
:1006100050524F4D000400436C6F736500000000A2
:100620000000000200456469740000000000000042
:10063000000000436C6561720000000000000020B3
:10064000005365742062617564000000004000532F
:1006500070656369616C00000000000000436C6F0E
:10066000736520616C6C0000000002526573746158
:100670007274000000000000010000000000000093
:100680000000000000000071776572747975696F71
:10069000700A6173646667686A6B6C0A077A7863CC
:1006A00076626E6D080A0B2C20202020202E0D0073
:1006B00051574552545955494F500A4153444647A2
:1006C000484A4B4C0A075A584356424E4D080A0BAB
:1006D0002C20202020202E0D000706001E001100D7
:1006E0000F0000002C002A001E0706001E00050057
:1006F0001E00000032002A002631323334353637EE
:100700003839300A21222324255E262A28290A5B2B
:100710005D3B27232D2B3D5F080A0B5C7C202020AE
:10072000202F0D0008070008081C1C3E2A7F367F7A
:100730002A7F3E7F003E08070018081C0C7E3E7F83
:100740003E7F0C7E081C001806060008001C002ACC
:1007500000080008000F00000000000000002A2B25
:100760002800000000000000000000000000000061
:100770000000000000002C9EB4A0A1A2A434A6A7F3
:10078000A5AE362D3738271E1F20212223242526EB
:10079000B333B62EB7B89F8485868788898A8B8CB9
:1007A0008D8E8F909192939495969798999A9B9C01
:1007B0009D2F3130A3AD350405060708090A0B0C3F
:1007C0000D0E0F101112131415161718191A1B1CE1
:1007D0001DAFB1B0B500080B000202020100090410
:1007E000000001020200000524001001052401019F
:1007F00001042402060524060001070581031000F8
:100800004009040100020A0000000705020240003E
:1008100000070583024000000403090412010002DE
:10082000EF020140412336800001010203014172C1
:100830006475696E6F204C4C430041726475626F41
:100840007900090B9EFF5EFFC2FFFAFFFAFFFAFF75
:10085000C2FF5EFF9EFF070707070607050703079E
:100860000507060707070707090BCFFFD7FF1BFF81
:10087000FDFFFEFFFDFF1BFFD7FFCFFF03070307B1
:100880000207020702070207020703070307050121
:100890000902A1010901A100850105091901290326
:1008A00015002501950375018102950175058103E8
:1008B00005010930093109381581257F750895032F
:1008C0008106C0C005010906A1018502050719E0DE
:1008D00029E7150025017501950881029501750824
:1008E00081039506750815002573050719002973FE
:1008F0008100C0080CFFFF02FE04FC08F890F0A085
:10090000E0C0C080800303020301010607090F0E47
:100910000E0000000000963511241FBECFEFDAE074
:10092000DEBFCDBF11E0A0E0B1E0E2EEFDE602C027
:1009300005900D92A435B107D9F729E0A4E5B1E0FF
:1009400001C01D92A83CB207E1F714E0CCE8D4E066
:1009500004C02197FE010E94E436CB38D107C9F7C5
:100960000E9410310C94EF360C9400006F927F922D
:100970008F929F92AF92BF92CF92EF92FF920F937E
:100980001F93CF93DF9300D01F92CDB7DEB75C01EA
:10099000F62EFC018484912CFFE18F1A910886EEDB
:1009A00091E09A838983992493949B822CE030E090
:1009B00042E050E0BE016F5F7F4FC5010E94322DC3
:1009C000CC24CA94E12C02EA12E0282D4CE050E03D
:1009D0006AE170E0C5010E948D2880EE91E09A8363
:1009E00089839B8225E130E042E050E0BE016F5FE9
:1009F0007F4FC5010E94322D01EA12E0282D45E10A
:100A000050E06AE170E0C5010E948D288BED91E015
:100A10009A8389839B822EE130E042E050E0BE0160
:100A20006F5F7F4FC5010E94322D00EA12E0282D32
:100A30004EE150E06AE170E0C5010E948D28F501A9
:100A400084852BEA829F212D1124269530E02A509F
:100A5000310987ED91E0A1E007E210E0AC016A2FD7
:100A6000C5010E94242B882331F01092A00210921D
:100A7000A1021092A202F501848590ED692E91E009
:100A8000792E8824839490E0880F991F63E070E0AA
:100A90000E94D0369B012F50310907E210E0682DEB
:100AA000A301C5010E94242B882339F08FEF809386
:100AB000A0028093A1028093A202F5E0FF1211C070
:100AC0002091A0028091A1029091A20233E834BD4E
:100AD000809587BD81EF809380002093880090935C
:100AE0008A000F900F900F90DF91CF911F910F917F
:100AF000FF90EF90CF90BF90AF909F908F907F909E
:100B00006F900895AF92BF92CF92EF92FF920F93A2
:100B10001F93CF93DF9300D01F92CDB7DEB75C0158
:100B2000F62E8091A3028823B9F088E892E09A8398
:100B3000898381E08B832CE030E045E050E0BE010A
:100B40006F5F7F4FC5010E94322D8091AF028111EE
:100B5000C6C01092A302B2C08091C009882399F048
:100B600083E792E09A83898311E01B8326E130E0DA
:100B700045E050E0BE016F5F7F4FC5010E94322DFE
:100B800081E692E016C08091B002882301F18AE4E8
:100B900092E09A83898311E01B8326E130E045E0EF
:100BA00050E0BE016F5F7F4FC5010E94322D87E389
:100BB00092E09A8389831B832DE130E045E050E089
:100BC000BE016F5F7F4FC5010E94322D77C080E26A
:100BD00092E0A1E00AE010E023E030E0AC016A2FEF
:100BE000C5010E94242B882391F0F50124852695C8
:100BF00080E490E0821B91099187808788E090E0F3
:100C00009387828781E08093A3020E9435168CE04F
:100C100092E0A1E006E110E023E030E0AC016A2FB1
:100C2000C5010E94242B882339F08091C0098111CD
:100C300003C081E08093C00980E092E09A838983B9
:100C400081E08B8322E230E043E050E0BE016F5F41
:100C50007F4FC5010E94322DF501248525538AE07E
:100C6000C82EEE24E3940CE719E043E250E062E37F
:100C700070E0C5010E948D288AEE91E0A1E00AE2B1
:100C800010E023E030E0AC016A2FC5010E94242B64
:100C9000882319F081E00E947C15F7E0FF1211C053
:100CA0008091A30281111092A3028091C009811149
:100CB0001092C00980E00E947C1533C087E0F816CE
:100CC000A1F389E0F81211C08091A302882349F1B1
:100CD000609149048BED98E00E94512322C0F7E017
:100CE000FF1609F3E9E0FE1699F3E5E0FE1219C0DC
:100CF0008091B0028823A9F00E94F215807380339E
:100D000071F48091A4028F5F8093A402803849F42B
:100D100080E00E947C1581E080931A0102C010924D
:100D2000A4020F900F900F90DF91CF911F910F9120
:100D3000FF90EF90CF90BF90AF9008952F923F9289
:100D40004F925F926F927F928F929F92AF92BF92DB
:100D5000CF92DF92EF92FF920F931F93CF93DF9387
:100D6000CDB7DEB727970FB6F894DEBF0FBECDBF65
:100D70003C01613009F0F6C0DC0118960D911C9120
:100D80001997065F1F4F1A964D905C901B97BAE01B
:100D90004B0E511CFC01848590E05C01FDE0AF1A14
:100DA000B108D3011D962C90312CB5E12B1A3108D6
:100DB00021E0220D41E04A0DB201C8010E94902EAF
:100DC0003FE5C32E32E0D32EE12CF12C420C531C14
:100DD0004CE2842E99249394C7016FE070E00E9446
:100DE000D036FB01E00FF11FFD83EC83D601ED91BE
:100DF000FD916D01EA0CFB1CC7016FE070E00E94E1
:100E0000D036CB01800F911F9F838E83D6012D9109
:100E10003C913097A9F0CF016AE070E00E94BC36A7
:100E2000685C7109629DC001639D900D729D900D7B
:100E30001124B4010E94BC36F201E61BF70B01C07D
:100E4000F20121153105A9F0C9016AE070E00E94A4
:100E5000BC36685C7109629DC001639D900D729DF6
:100E6000900D1124B4010E94BC369201261B370B51
:100E700001C092014E815F81BF018C819D810E94E2
:100E8000C02EEDE7F2E0EC15FD0509F0A5CF00E07E
:100E900010E0E12CF12C8DEF882E99249A9493E0A8
:100EA000A92EB12C24E6C22ED12CD30118968D91F7
:100EB0009C91199702969093860480938504C701AC
:100EC000B4010E94D036640D751D70938404609344
:100ED0008304C801B5010E94BC36CB0188539F4FE3
:100EE000B6010E94D036CB010E94062CE20CF31C06
:100EF000045D1E4F003BB4E01B07B9F600917D0274
:100F000010917E02F3018485869560857185680F56
:100F1000711D68517109858542855385480F511DA2
:100F20004850510988EB91E09A83898381E08B8353
:100F300020E0CE0101960E941815C80168EE73E00A
:100F40000E94BC368C01CB010E94062C60E08EE230
:100F50000E943513C8010E94062C60E086E50E94BD
:100F6000351338C06530B1F580915E0281112FC014
:100F70008EE50E94A6159C0140E050E060E070E321
:100F800081E190E00E947B36EFE5F2E08DE792E0B0
:100F900042815381419351938E179F07C9F7203D9A
:100FA000F7E03F0738F0293883E1380728F028E8D0
:100FB00033E102C020ED37E030937E0220937D02C2
:100FC0008CE380935E0281E080931A0103C081501C
:100FD00080935E0260E270E0C3010E949F29882333
:100FE00049F0EFE5F2E08FE792E0119211928E174F
:100FF0009F07D9F727960FB6F894DEBF0FBECDBF77
:10100000DF91CF911F910F91FF90EF90DF90CF90E4
:10101000BF90AF909F908F907F906F905F904F9018
:101020003F902F9008952F923F924F925F926F9230
:101030007F928F929F92AF92BF92CF92DF92EF9268
:10104000FF920F931F93CF93DF93CDB7DEB729970E
:101050000FB6F894DEBF0FBECDBF8C01613009F032
:10106000DCC0DC011896ED90FC901997BAE0EB0E0D
:10107000F11CFC0162847384FAE06F0E711CDC01C8
:101080001C968C911C9790E0FC013D97FD83EC83AE
:101090001D964C90512CF5E14F1A510821E0240D7A
:1010A0004E2F4F5FB301C7010E94902E20E8A22E61
:1010B00022E0B22EC12CD12C3FE0232E312C640C27
:1010C000751C4EEC842E99249A94C601B1010E949D
:1010D000D036FB01EE0DFF1DFF83EE83D501ED91B0
:1010E000FD915D012C813D81C20ED31EC601B1016F
:1010F0000E94D036CB018E0D9F1D99878887D50120
:101100002D913C91309771F04E9EC0014F9E900DF5
:101110005E9E900D1124B4010E94D036FB01E60DB5
:10112000F71D01C0F3012115310571F0429EC00188
:10113000439E900D529E900D1124B4010E94D03612
:101140009B01260D371D01C0930148855985BF01BC
:101150008E819F810E94C02EBEE9AB16B2E0BB0615
:1011600009F0B3CFE12CF12CC12CD12C8DEF882EBE
:1011700099249A9493E0A92EB12CF8018085918549
:1011800002969093860480938504C601B4010E9460
:10119000D036660D771D7093840460938304C70175
:1011A000B5010E94D036CB010E94062CC40CD51C80
:1011B000F2E3EF0EF11C28ECE216F104F1F6D8018F
:1011C0001C968C911C97869518966D917C91199719
:1011D000680F711D685171091D968C911D971A96A3
:1011E0004D915C911B97480F511D4850510982EC5D
:1011F00091E09A83898381E08B8320E0CE01019680
:101200000E94181580919E0290919F020E94062CC8
:1012100060E083E40E9435132DC0653059F580915C
:101220007F02811124C0E0E8F2E082819381819302
:101230009193B2E0EE39FB07C1F787EC0E94A61547
:101240008851914097FD06C0833391052CF082E3CD
:1012500090E002C080E090E090939F0280939E0215
:101260008CE380937F0281E080931A0103C0815058
:1012700080937F0260E270E0C8010E949F2988236A
:1012800049F0E0E8F2E080EA92E0119211928E17C4
:101290009F07D9F729960FB6F894DEBF0FBECDBFD2
:1012A000DF91CF911F910F91FF90EF90DF90CF9042
:1012B000BF90AF909F908F907F906F905F904F9076
:1012C0003F902F9008952F923F924F925F926F928E
:1012D0007F928F929F92AF92BF92CF92DF92EF92C6
:1012E000FF920F931F93CF93DF93CDB7DEB727976E
:1012F0000FB6F894DEBF0FBECDBF9F838E83162F2F
:10130000DC011A96CD90DC901B9720900301309061
:1013100004013101B1E06B2277244AE750E06CE52B
:1013200072E00E94ED268091A7028F3F61F0E0E11C
:101330008E9FC00111248951974F2E813F8128171C
:10134000390709F454C1113009F0C9C0E0905C02BA
:10135000F0905D0283E0EE0CFF1C8A95E1F7369475
:101360002794560139E0A30EB11CC601C3969C8395
:101370008B83C301A1E08A27B82FB170BD832501FB
:10138000EFEF4E1A5E0AAE81BF8118968D909C9049
:101390001997C40102969093860480938504509215
:1013A00084044092830460E08F2D82958F700E94A8
:1013B000101560E08F2D0E94101560E0C70104E059
:1013C000969587950A95E1F70E94101560E08E2D9D
:1013D0000E9410156401B6E1CB0ED11CF401EA584D
:1013E000FF4FFA83E9834701C4010E947A15182F41
:1013F000D0928604C0928504509284044092830463
:1014000028143904B9F400E027E044E0B501C6012E
:101410006114710411F0049601C001970E94D01567
:10142000D0928204C09281045092800440927F0442
:101430006D8101C060E0812F82958F700E94101530
:101440002814390421F461E06114710409F460E0A6
:10145000812F0E941015FCE0CF0ED11C2FEF821AB5
:10146000920A89819A81C816D90609F0BDCF98E001
:10147000E90EF11CA7E0AA0EB11CEB81FC81EA1574
:10148000FB0509F07CCFAE81BF811D964C911D9765
:1014900049501A966D917C911B97675F7F4F189604
:1014A0008D919C91199720E0449627960FB6F89459
:1014B000DEBF0FBECDBFDF91CF911F910F91FF9087
:1014C000EF90DF90CF90BF90AF909F908F907F90E4
:1014D0006F905F904F903F902F900C94BE2A1230E7
:1014E00009F05BC0E0917009F0E0AE81BF81189611
:1014F0008D919C911997E81BF90BCF0145978F357A
:10150000910508F0BBC02091720930E01A968D91C8
:101510009C911B97281B390B2A5031092A3231051F
:1015200008F0ACC0CF0144976CE070E00E94D03668
:101530007B0160915C0270915D02A3E0660F771FF2
:10154000AA95E1F7CB018E0D9F1D9A838983C9016E
:1015500067E070E00E94D036B3E0660F771FBA955F
:10156000E1F729813A81620F731F660F771F8CE0C4
:101570008E9D90018F9D300D1124265E3F4F81E09E
:1015800090E02E173F0714F080E090E0680F791F7D
:10159000709304016093030126C0193009F06EC0F6
:1015A0008091490430ED380F39833A3038F19FE9A2
:1015B000980F963010F4875506C09FEB980F963021
:1015C00008F05CC08753898319C0A90163E0440F08
:1015D000551F6A95E1F78417950708F44AC03093C0
:1015E0005D0220935C0281E080931A0147C084EA87
:1015F00091E09093060180930501A5CE369427943F
:10160000C1010E947A15672821F0682F607F8981C7
:1016100006C08F70A98190E1A99FB0011124682BA9
:10162000C1010E94EC238091030190910401811576
:10163000B8E09B07C0F601969093040180930301E4
:101640009695879520915C0230915D02A9014A5FD1
:101650005F4FE3E0440F551FEA95E1F7B9016F5F73
:101660007F4F8417950708F4B0CF485F5F4F9B0109
:10167000F5CF2150310948505109ADCF27960FB60B
:10168000F894DEBF0FBECDBFDF91CF911F910F91B8
:10169000FF90EF90DF90CF90BF90AF909F908F9092
:1016A0007F906F905F904F903F902F9008952F9272
:1016B0003F924F925F926F927F928F929F92AF92E2
:1016C000CF92DF92EF92FF920F931F93CF93DF930E
:1016D000CDB7DEB727970FB6F894DEBF0FBECDBFEC
:1016E0004C01162FFC01C180D280F8EBCF16F2E03E
:1016F000DF0659F082EE90E09A83898381E08B8344
:101700002AE532E03D832C8307C0DA82C9821B823E
:1017100048E552E05D834C83F401248530E03901D3
:10172000FCE06F1A7108F401858590E0AC014C5023
:1017300051095F834E83CA0167E070E00E94D03692
:101740002B01130177FE04C0190159E0251A310855
:101750003594279435942794B101CE0101960E94C7
:1017600077114816590624F4AC014419550902C0F2
:1017700040E050E06C817D81C4010E94ED26113073
:10178000E1F5EC81FD81E080F180F4014285538533
:1017900060857185F8EBCF16F2E0DF0679F0455FE2
:1017A0005F4F6E5F7F4FA12CCC24CA94DC2C0E813E
:1017B000262DCE0101960E94772DC2C18091A702ED
:1017C0008F3F59F020E1829FC00111248951974F2A
:1017D000AA24A3948816990609F0A12CC0900101AF
:1017E000D0900201455F5F4F6E5F7F4F0E81262DC7
:1017F000CE0101960E94772D06C038EBC31632E069
:10180000D30609F09DC180E190E00E947A158435ED
:1018100001F161E070E0C4010E949F29882309F46E
:1018200047C064E580E190E00E94EC236FE481E131
:1018300090E00E94EC2363E582E190E00E94EC23BB
:1018400068E483E190E00E94EC2334E1E32EF12C84
:1018500013C081E190E00E947A158F34D1F682E1C5
:1018600090E00E947A158335A1F683E190E00E9412
:101870007A15883471F644C1670134E1C31AD1087E
:10188000CE0101960E946011C816D9066CF4B6010B
:10189000CE0101960E94C211682FC7010E94EC235D
:1018A0004FEFE41AF40AE8CF60E0C7010E94EC238E
:1018B00060E270E0C4010E949F29811110C0CE0136
:1018C00001960E946011209101013091020182175E
:1018D000930768F4909302018093010108C0E8EB3C
:1018E000F2E0119254E0E834F507D9F7E8CF193067
:1018F00009F089C010914904183011F500910101D7
:10190000109102010115110509F448C00150110997
:101910007801CE0101960E9460119C01E216F30647
:1019200054F4E981FA81EE0DFF1D918190838FEFD0
:10193000E81AF80AF3CF10930201009301012EC0B8
:10194000CE0101960E9460118039E1E09E0734F5D6
:101950002091010130910201BC0149815A81261771
:10196000370754F4DA01A60FB71FFD013197E08164
:10197000EC9361507109F1CFFA01E20FF31F10836C
:101980008217930729F4E981FA81E20FF31F11828C
:101990002F5F3F4F3093020120930101CE0101964A
:1019A0000E9460117C0180E090E000E010E08E1564
:1019B0009F0584F4A101BC01CE0101960E94591C2F
:1019C00020910101309102012817390718F00F5FAB
:1019D0001F4FEDCFEC81FD8120813181C801841939
:1019E00095098217930720F001969183808307C0A1
:1019F0000217130720F4EC81FD811183008381E03D
:101A000080931A019DC0123009F09AC0409070096D
:101A1000512CF40180859185481A590AF2E04F1A39
:101A200051088091720990E0F40122853385821B70
:101A3000930B0B9757FC84C097FD82C04614570444
:101A40000CF07EC02E813F81821793070CF078C086
:101A500067E070E00E94D0367B01EC81FD8100815F
:101A60001181CE0101960E9460113C01812C912CC4
:101A7000861497046CF40115110551F0A101B4010D
:101A8000CE0101960E94591C4C0101501109F0CF62
:101A9000CE0101960E9460118C01612C712C801680
:101AA00091060CF04DC0A101B401CE0101960E9437
:101AB000591C6E147F04F9F4559447945594479437
:101AC0009C0128193909421653063CF4480C591C4C
:101AD000509202014092010192CF0817190729F490
:101AE00010930201009301018ACF019790930201A4
:101AF0008093010184CFFFEF6F1A7F0A4C01CFCF93
:101B000068E070E0C4010E949F29811103C0163073
:101B100009F07FCE48EBC42E42E0D42E54E1E52EEE
:101B2000F12CC7010E947A15F60181936F01FFEF36
:101B3000EF1AFF0A24EAE21621E0F20691F769CED5
:101B400027960FB6F894DEBF0FBECDBFDF91CF91C1
:101B50001F910F91FF90EF90DF90CF90AF909F90EB
:101B60008F907F906F905F904F903F902F9008954F
:101B70006F927F928F929F92AF92BF92CF92DF929D
:101B8000EF92FF920F931F93CF93DF9300D01F929A
:101B9000CDB7DEB74C01B62E88E591E09A838983F4
:101BA0001B82D4011C968C9190E07C01BFE0EB1A63
:101BB000F108F7FE04C07C01ECE0EE1AF108F594A0
:101BC000E794F594E794D4011D968C9190E00C97DE
:101BD00067E070E00E94D0366B01B701CE0101963C
:101BE0000E9477118C0160E270E0C4010E949F297D
:101BF000882359F0E8E5F1E01192B2E0E835FB07FF
:101C0000D9F7109257011092560164E070E0C401B8
:101C10000E949F2981110FC060E470E0C4010E94FE
:101C20009F298823D1F040E050E068E47FE082E023
:101C30000E94562512C0612C712CC3010E947A1596
:101C4000682F8AE898E00E94AF1DEFEF6E1A7E0AB7
:101C50006114F4E07F0689F7DFCFC016D1061CF4CB
:101C60000C191D0902C000E010E0A80164E571E054
:101C7000C4010E94ED2629E0B21207C06091490418
:101C80008AE898E00E94AF1DF1C081E0B8122BC035
:101C90008091A7028F3F59F0A0E18A9FC0011124D3
:101CA0008951974FAA24A3948816990609F0A12C6C
:101CB000CE0101960E946011E0905401F090550110
:101CC000F40105850C5024852F5042855385455FCE
:101CD0005F4F608571856E5F7F4F6C01CE0101960D
:101CE0000E94772DC3C0F5E0BF12C0C0B12C8AE0BE
:101CF000982E8AE898E00E94CA1D892B09F498C0A2
:101D00008AE898E00E940A1F882EA0905601B090A1
:101D100057012FEFA216B10459F5A70160E070E05A
:101D2000CE0101960E94591CF501E81BF90BF093B6
:101D30005701E0935601AC01485A5E4F88E591E0A7
:101D40009C0128553140E217F3073CF0DA012D9150
:101D5000AD01DC012D93CD01F3CFE85AFE4FCF0149
:101D6000885591408F3F910509F014F41192F7CFF7
:101D7000B8E08B1619F0EFE78E1214C0809156016F
:101D800090915701181619061CF0BB24B394B1CFDB
:101D900001979093570180935601FC01E85AFE4F3A
:101DA0001082F3CFFAE08F1219C080915601909102
:101DB00057011816190634F4FC01E95AFE4F208128
:101DC0002D30A1F19C012F5F3F4F3093570120939D
:101DD0005601FC01E85AFE4F9082D7CF2BE18212C8
:101DE00012C08AE898E00E940A1F8B3571F68AE8D3
:101DF00098E00E940A1F80538A3038F68AE898E0FB
:101E00000E940A1FC2CF80EE880D8F3508F0BDCF2B
:101E100080915601909157019C012F5F3F4F309365
:101E2000570120935601FC01E85AFE4F8082ADCF46
:101E3000BB20E1F00115110539F08091540190911A
:101E400055010817190779F4B701CE0101960E94D0
:101E50007711C816D9061CF48C010C191D091093B2
:101E600055010093540181E080931A010F900F9067
:101E70000F90DF91CF911F910F91FF90EF90DF9026
:101E8000CF90BF90AF909F908F907F906F9008956C
:101E90009F92AF92BF92CF92DF92EF92FF920F93F9
:101EA0001F93CF93DF9300D01F92CDB7DEB77C0195
:101EB00080E6F701848780E3858780E190E0918761
:101EC000808788E090E09387828787ED90E09A830F
:101ED000898381E08B8326E030E046E050E0BE015C
:101EE0006F5F7F4FC7010E94322D8BE1A82E81E0EA
:101EF000B82ED12C0EE010E0CC24C3949BE0992E98
:101F0000F70120853185C901069662857385600FCA
:101F1000711F40916809413061F4209100012D1139
:101F200003C04AEB50E002C04CEA50E00E945E2C35
:101F30001EC04230E1F44091700950E04817590743
:101F4000B4F08091720990E08617970784F02A5DBB
:101F50003F4F241735075CF06A5F7F4F681779079A
:101F600034F0D0920001C0921A01909268098091D9
:101F700068098130B1F4F50180819181F7012285F2
:101F80003385408551854E5E5F4F50938604409364
:101F90008504200F311F30938404209383040E9412
:101FA000062C095F1F4FF2E0AF0EB11CD3940A322A
:101FB000110509F0A5CFF701058510E00B511109B6
:101FC000248530E0245231098FEC90E0A1E0AC018F
:101FD0006A2FC7010E94242B882359F081E0809347
:101FE00000010E94B32A8FEF9FEF90939708809390
:101FF0009608F701058510E000511109248530E0AD
:102000002452310988EC90E0A1E0AC016A2FC701AD
:102010000E94242B882359F00E94B32A8FEF9FEF50
:102020009093970880939608C7010E9498250F9077
:102030000F900F90DF91CF911F910F91FF90EF9034
:10204000DF90CF90BF90AF909F900895CF93DF9394
:10205000EC019C01235F3F4FF90185919491892BFD
:10206000A9F0F90145915491E7EEF8E080E090E0A5
:102070006081662329F06181728146175707B1F0AC
:10208000019670968830910599F721C0FE013B9624
:1020900045915491E7EEF8E080E090E0608166239E
:1020A00089F0638174814617570761F444E0880F13
:1020B000991F4A95E1F78951974F009741F00E9487
:1020C0002A253AC0019670968830910539F7F901B2
:1020D00045915491FE013B966591749183E00E9475
:1020E0005625DC01892B41F1CE01029616969C9370
:1020F0008E93159781E017968C931797FE013F9664
:10210000E491F0E01996FC93EE931897FE01709617
:10211000E491F0E01B96FC93EE931A97FE01719602
:10212000E4911C96EC931C97FE017296E4911D9627
:10213000EC931D97CD0102C080E090E0DF91CF913C
:1021400008957F928F929F92AF92BF92CF92DF922B
:10215000EF92FF920F931F93CF93DF9300D01F92C4
:10216000CDB7DEB74C01FC01E180F2809AE0A92EE8
:10217000B12C2EE0C22ED12C77247394F7018591D7
:102180009491892B09F43BC0C70102969A838983F5
:102190007B82F7016591749185019601AE014F5FD5
:1021A0005F4FC4010E94DF298823B1F0C7010E945C
:1021B00026108C01009781F00E9418258983BE01AA
:1021C0006F5F7F4F85E00E94531685E08C0DF8010C
:1021D000868785E08A0D8787FEE1CF0ED11CF4014A
:1021E000848590E0C816D90634F0F6E1AF0EB11C34
:1021F0008EE0C82ED12C83E1E80EF11CBFCF0F90EA
:102200000F900F90DF91CF911F910F91FF90EF9062
:10221000DF90CF90BF90AF909F908F907F90089568
:10222000EF92FF920F931F93CF93DF9300D01F92F3
:10223000CDB7DEB77C0162E070E00E949F298DED92
:1022400094E09A83898381E08B830AE010E02CE696
:1022500030E0AE014F5F5F4F69EF74E0C7010E944D
:10226000DF298823A9F08AEC94E00E9426108C01D3
:10227000009771F00E9418258983BE016F5F7F4F20
:1022800085E00E94531681E7F80186878FE08787F3
:102290000F900F900F90DF91CF911F910F91FF90B2
:1022A000EF900895DC0112962C911297ED91FC911C
:1022B000E60FF71F213011F484910895808108956D
:1022C000FC01A081B181109779F08281813019F4ED
:1022D000CD010C945C36FD0101900020E9F73197A7
:1022E000CF018A1B9B0B089580E090E008956F92C8
:1022F0007F928F929F92AF92BF92CF92DF92EF9296
:10230000FF920F931F93CF93DF934C013B010E94E9
:1023100060117C0100E010E0C0E0D0E06C0181E0E1
:10232000C81AD1080E151F05ECF45E018FEFA81A2C
:10233000B80AA301B801C4010E94591C8C01E81617
:10234000F90671F4B601C4010E9452118A3031F0CD
:10235000B601C4010E9452118D3011F42296E2CFD1
:10236000E501E0CFCE01DF91CF911F910F91FF905A
:10237000EF90DF90CF90BF90AF909F908F907F9025
:102380006F9008950F931F93CF93DF9377FD0FC046
:10239000EB018C010E946011C817D90744F4BE01FB
:1023A000C801DF91CF911F910F910C94521180E0E1
:1023B000DF91CF911F910F910895CF93DF9300D0BC
:1023C0001F92CDB7DEB79A83898381E08B83CE01DC
:1023D00001960E94601121E0892B09F020E0822FF4
:1023E0000F900F900F90DF91CF9108950C96FC0104
:1023F0002591349181E0232B09F080E008950F931B
:102400001F93CF93DF93EC018B010E94F611882379
:1024100061F02E96CE010E94F611811117C0CE01F7
:102420000E94DD11811112C00AC02C96FE01859117
:1024300094910823192381E0012B49F407C0B801C6
:10244000CE010E94FF11882321F301C080E0DF91BB
:10245000CF911F910F910895EF92FF920F931F93C9
:10246000CF93DF937B01EC012E9600E010E0CE01CC
:102470000E94F61181110FC0CE010E94DD11811161
:102480000AC0B701CE010E94FF11882311F00F5F2F
:102490001F4F2E96ECCFC801DF91CF911F910F9166
:1024A000FF90EF9008950F931F93CF93DF936115E3
:1024B0007105D1F06817790711F481E016C08B011E
:1024C000EC010E94F611882379F02E96CE010E942D
:1024D000F611811109C0CE010E94DD11811104C0E5
:1024E0000C171D0791F7E9CF80E0DF91CF911F9185
:1024F0000F9108954F925F926F927F928F929F9269
:10250000AF92BF92CF92DF92EF92FF920F931F9301
:10251000CF93DF9300D01F92CDB7DEB70E941B246C
:102520004C010FED15E09AE0C92ED12C552453949F
:1025300027E0422E37E0632E712CC8010E94DD1186
:10254000811135C0C8010E94F611882369F1B401D8
:10255000C8010E94FF11882339F11A8309835B8225
:10256000CE0101960E94601101965C01AA0CBB1C71
:10257000AA0CBB1C8091700990E08C159D0534F06D
:1025800096012A0D3B1D82179307A4F060917704F2
:1025900070917804C8010E945312811110C086E026
:1025A000A80EB11CCA0CDB1C025F1F4FC6CF80E017
:1025B00090E047C080917209883040F741C0C8015F
:1025C0000E94F611882331F0B401C8010E942C1238
:1025D0009C0102C020E030E08091700990E08C15F1
:1025E0009D05ECF2A6014D5C5F4F48175907BCF200
:1025F00080917209893098F290E0429EA001439E3A
:10260000500D1124465F5F4F8417950744F60897D5
:10261000B3010E94D0367B01621773078CF4F7FC7C
:10262000BECF025F1F4FB401C8010E94FF11882373
:10263000B1F3E114F10421F081E0E81AF108EFCFE1
:10264000C8010F900F900F90DF91CF911F910F91C4
:10265000FF90EF90DF90CF90BF90AF909F908F90C2
:102660007F906F905F904F9008952F923F924F927E
:102670005F926F927F928F929F92AF92BF92CF9212
:10268000DF92EF92FF920F931F93CF93DF93CDB71B
:10269000DEB729970FB6F894DEBF0FBECDBF8052CC
:1026A000813608F0A4C16887282F30E0220F331F3D
:1026B000F901E15EFA4F9491F901E05EFA4F24913D
:1026C00029870091830410918404A8014F5F5F4F14
:1026D0004A012091850430918604592F5074252E8B
:1026E000892F8072382EA8014E5F5F4F5A01592FF3
:1026F0005071452E892F8870582E492F4470642EB2
:10270000A8014D5F5F4F6A01592F5270752E892FB6
:1027100081708983498542704A83A8014C5F5F4F6D
:102720007A01598550745B83898580728C834985D1
:1027300040714D83598558705E83898584708F837D
:10274000498540FFA6C097FF05C0462FB401C901C7
:102750000E940024222049F08091850490918604F3
:102760004885B40101960E940024332049F08091ED
:102770008504909186044885B40102960E94002445
:10278000442041F04885B5018091850490918604EC
:102790000E940024552049F0809185049091860480
:1027A0004885B50101960E940024662049F0809179
:1027B0008504909186044885B50102960E94002404
:1027C000772041F04885B601809185049091860478
:1027D0000E9400245981552349F0809185049091ED
:1027E00086044885B60101960E9400248A818823C8
:1027F00049F080918504909186044885B60102963F
:102800000E940024298527FF08C04885B7018091D0
:102810008504909186040E9400243B81332349F073
:1028200080918504909186044885B70101960E94A5
:1028300000244C81442349F08091850490918604C2
:102840004885B70102960E9400240B5F1F4F5D81EF
:10285000552341F04885B801809185049091860404
:102860000E9400248E81882349F0809185049091F4
:1028700086044885B80101960E9400242F812223F6
:1028800009F4ACC080918504909186044885B80114
:10289000A2C097FF05C04885B801C9010E94002465
:1028A000222049F080918504909186044885B801E2
:1028B00001960E940024332049F080918504909174
:1028C00086044885B80102960E940024442041F005
:1028D0004885B40180918504909186040E9400246B
:1028E000552049F080918504909186044885B40173
:1028F00001960E940024662049F080918504909101
:1029000086044885B40102960E940024772041F095
:102910004885B50180918504909186040E94002429
:102920003981332349F0809185049091860448854C
:10293000B50101960E9400244A81442349F0809108
:102940008504909186044885B50102960E94002472
:10295000598557FF08C04885B6018091850490913C
:1029600086040E9400248B81882349F0809185048D
:10297000909186044885B60101960E9400242C811E
:10298000222349F080918504909186044885B60100
:1029900002960E9400243D81332341F04885B7010F
:1029A00080918504909186040E9400244E814423E6
:1029B00049F080918504909186044885B70101967D
:1029C0000E9400245F81552349F0809185049091F5
:1029D00086044885B70102960E94002480918504F0
:1029E000909186040496909386048093850429969A
:1029F0000FB6F894DEBF0FBECDBFDF91CF911F9110
:102A00000F91FF90EF90DF90CF90BF90AF909F908D
:102A10008F907F906F905F904F903F902F90089590
:102A20008F708A3010F4805D01C0895C0C9435137E
:102A3000EF92FF921F93CF93DF937C01122F70933D
:102A4000860460938504509384044093830460E07B
:102A500070E0EB012196C7010E94C211882329F082
:102A6000612F0E943513BE01F4CFDF91CF911F91EA
:102A7000FF90EF900895EF92FF921F93CF93DF9313
:102A800000D01F92CDB7DEB77C01162F6130B1F4B4
:102A900049EF54E06AE170E081E190E00E945E2C31
:102AA00085EE94E09A8389831B8320E04DE150E01A
:102AB0006FE170E0CE0101960E94181580916E09B9
:102AC000813478F0C7010E94982540E050E060E131
:102AD00071E181E00E945625FC0113861286118661
:102AE00010860F900F900F90DF91CF911F91FF9064
:102AF000EF9008950C946536CF939091B00298179B
:102B000019F1C82F81111EC068ED8BED98E00E946D
:102B1000062367ED8BED98E00E9406236AED8BEDAE
:102B200098E00E94062369ED8BED98E00E94062351
:102B300060E88BED98E00E94062360EB8BED98E057
:102B40000E940623C093B002CF9108959091640033
:102B50009E7F9093640080937C00873C11F480E218
:102B600003C080917B008F7D80937B0062E070E0EA
:102B700080E090E00E948C3080917A0080648093A5
:102B80007A0080917A0086FDFCCF20917800309108
:102B9000790090916400916090936400C901089558
:102BA000CF92DF92EF92FF920F931F93CF93DF9319
:102BB0007B01122FEC016C01C40ED11CCC15DD057C
:102BC00044F4202F412FB701CE010E94BE2A219646
:102BD000F5CFDF91CF911F910F91FF90EF90DF9094
:102BE000CF900895CF930E94E42383FF02C0C0E1F9
:102BF00001C0C0E00E94E42382FDC0620E94E42381
:102C000087FDC4600E94E42384FDC8600E94E42321
:102C100085FDC1600E94E42386FDC2608C2FCF91A8
:102C200008959C0180E090E0F901E80FF91F4491BC
:102C3000442329F0E491EA3011F00196F5CF08958C
:102C4000CF93C09189040E9418259C2FCF9108959D
:102C5000FC019081DB018C91981305C081E02181FA
:102C600011969C91291380E00895CF9387E896E010
:102C70009093060180930501C1E0C093AF020E94CA
:102C8000F21580936709C0931A01CF91089590912E
:102C90006909981307C0109269098FEF80936C0936
:102CA00080936D0908959091690991110BC08093EB
:102CB0006909FB018081918190936D0980936C0972
:102CC00010926E090895FF920F931F93CF93DF9395
:102CD00000D0CDB7DEB78C01F62EDC018C918330AD
:102CE000D9F5B2E06B132EC0F801228533858091AF
:102CF000720990E0A901495F5F4F4817590714F125
:102D0000281739070CF07BC02091700930E08085CE
:102D10009185AC014B5F5F4F421753070CF06FC0BA
:102D20000996821793070CF46AC0C8010E941825FF
:102D30008983BE016F5F7F4F82E00E94531681E05E
:102D400080931A0162E070E0C8010E949F298823E5
:102D500019F0C8010E949825809169098330B9F55E
:102D6000F4E0FF122DC0D8011A968D919C911B970B
:102D700020917A0930917B09280F391F28303105BD
:102D800044F428E030E0281B390B30937B09209372
:102D90007A09F801408551852091780930917909A7
:102DA000240F351F3187208720917A0930917B09C4
:102DB000820F931F9387828781E080931A0112C04C
:102DC000F3E0FF120FC083E00E9447160BC0823071
:102DD00049F483E0F81206C082E00E944716C80159
:102DE0000E94982510928904D8011396ED91FC91C8
:102DF0001497309779F06F2DC80109950BC0C80161
:102E00000E9418258983BE016F5F7F4F83E00E9477
:102E1000531698CF0F900F90DF91CF911F910F9184
:102E2000FF9008952F923F924F925F926F927F9200
:102E30008F929F92AF92BF92CF92DF92EF92FF92CA
:102E40000F931F93CF93DF93CDB7DEB72B970FB6BA
:102E5000F894DEBF0FBECDBF182F80936809853070
:102E600099F407EE18E0F8018081882321F065E0ED
:102E7000C8010E946316005F1F4FF9E007361F0765
:102E800091F70E942B24F6C1813001F50FEA12E080
:102E900057EAE52E52E0F52EF80182918F018F3F1F
:102EA00041F0F0E18F9FC00111248951974F0E949A
:102EB000C525E016F10681F70E942B240E941B24F1
:102EC0006C010FED15E0E12CF12C87C0823009F088
:102ED00057C08091720990E02091700930E0A7EA14
:102EE000B2E04FEAE42E42E0F42E0D910F3F09F4D8
:102EF00091C140E1049F80011124F801E951F74F8D
:102F000060857185261737078CF0428553858417B5
:102F1000950764F0D4846D0D711D2617370734F4BE
:102F20006585460F511D8417950754F0F801E95146
:102F3000F74F4081413021F0EA16FB06B1F66AC135
:102F40000951174F0115110509F464C1E091A70259
:102F5000E83070F480E1E89FF0011124E951F74F67
:102F60008081823029F4F8018081823009F052C1D9
:102F7000C8010E942A2562E0C8010E9463164AC166
:102F800080916909882371F080916C098F3F51F01D
:102F9000F0E18F9FC0011124612F8951974F0E944A
:102FA0006316A9C1E7EAF2E081918F3F51F020E179
:102FB000829FC0011124612F8951974F0E9463168F
:102FC00050C132E0EF3AF30779F74BC1C8010E94D4
:102FD000F611811108C0025F1F4FC8010E94DD1168
:102FE0008823A1F307C0B601C8010E94FF11811117
:102FF0005CC1F1CFEF2809F43DC10E941B242C01D4
:103000008091AF02882341F0C0907904D0907A0477
:10301000D194C194D10802C0C12CD12C01E027E089
:1030200040E8B60180E090E00E94D01520E042E048
:10303000B60180E090E00E94BE2A40E0B60181E047
:1030400090E00E94002420E042E0B6018FE790E08B
:103050000E94BE2A40E0B6018EE790E00E94002464
:1030600040E8B601695F7F4F80E090E00E941E2B30
:103070009FEDE92E95E0F92E2AE0A22EB12C11E069
:1030800096012F5F3F4F39872887160138E0230EBE
:10309000311CC60109969B878A87C7010E94DD11F2
:1030A0008111E8C0C7010E94F611882309F4AEC05F
:1030B000B201C7010E94FF11882309F4A7C06091E3
:1030C000770470917804C7010E945312982EFA82F7
:1030D000E9821B83CE0101960E9460110196FC01DA
:1030E000EE0FFF1FEE0FFF1FFD83EC83992049F0C9
:1030F00000E028E04C81B601C5010E94D01521E016
:1031000001C020E0FA82E9821B8348855985B50118
:103110006E5F7F4FCE0101960E941815992009F429
:1031200070C0C7010E94F611882331F0B201C701B7
:103130000E942C123C0102C0612C712CF7E0F69D1C
:103140004001F79D900C112422E0820E911C01E0B9
:10315000282D44E3B101C5010E94D015282D44E378
:10316000B101C5010E94902E20E0482D6A857B8523
:10317000C501C4960E94BE2AB401620D731D44E3CA
:10318000C50101960E941E2B46013AE0830E911C58
:10319000C50106969F838E831614170494F59EE04E
:1031A000E90EF11CB201C7010E94FF118823A1F3AF
:1031B000E1E06E1A71086091770470917804C7019C
:1031C0000E945312882371F000E028E044E3B40128
:1031D00062507109C5010E94D015FA82E9821B83F1
:1031E00021E004C0FA82E9821B8320E0A4016E8101
:1031F0007F81CE0101960E941815F7E08F0E911C79
:10320000CBCF8C819D810696A80EB91E2EE0E20ED2
:10321000F11C43CFE091A702E83048F430E1E39F8E
:10322000F0011124E951F74F8081823019F10E9499
:103230007A129093780480937704892BD9F08FEFDA
:1032400089838A83BE016F5F7F4F88E00E94531697
:1032500004C0109378040093770481E080931A01EE
:1032600009C0183009F047C0E0917704F091780464
:103270003097F9F4109268092B960FB6F894DEBFD8
:103280000FBECDBFDF91CF911F910F91FF90EF90B7
:10329000DF90CF90BF90AF909F908F907F906F9076
:1032A0005F904F903F902F9008954FEFE41AF40AEB
:1032B00092CE3C9685919491811541E0940751F00E
:1032C00081159240B9F607EE18E037E6E32E39E0B3
:1032D000F32E09C0E0E0F0E00995CCCF005F1F4F6E
:1032E000E016F10639F2F80180818330B9F7C801A0
:1032F0000E949825F3CF143039F580916909883000
:1033000009F0B8CF0E947A122091770430917804A6
:10331000009789F4C9010E94F6118111ABCF009189
:10332000770410917804C8010E94F611811191CFA1
:103330000E501109F8CF8217930709F49BCF909391
:1033400078048093770489CF133009F093CF80916C
:103350006909883009F08ECF0E947A129093780420
:1033600080937704009721F00E94F611882359F08A
:1033700088E00E94471681E080931A011092780439
:103380001092770477CF88E00E941217F1CF2F9226
:103390003F924F925F926F927F928F929F92AF92E5
:1033A000BF92CF92DF92EF92FF920F931F93CF9332
:1033B000DF93CDB7DEB72F970FB6F894DEBF0FBE01
:1033C000CDBF8B870E94F215982E9091AF0284FF9B
:1033D0001FC08091670984FD1BC08091B0028111DC
:1033E00017C08091C009882331F01092C00981E094
:1033F00080931A010DC081E089278093AF0281116B
:103400000E94351681E080931A019092670938C2B4
:10341000992309F4EBC1A0900501B0900601C50104
:103420000E9411169C838B839C01E3E0220F331FC3
:10343000EA95E1F7A9014C5F5F4F59874887CA01B8
:1034400057FD019695958795919581959109FC0178
:10345000E05CFF4FFE83ED837C01FEE3EF0EF11C89
:1034600001E022E248856FE170E0C7010E94D015BB
:1034700022E248856FE170E0C7010E94902EC501ED
:103480000E9411161C012B813C81281B390B220F35
:10349000331F220F331F4D815E81240F351F3F875D
:1034A0002E8760904B0470904A0490FE0AC0809171
:1034B000670980FD06C0662021F08FEF860D80939E
:1034C0004B0491FE09C08091670981FD05C0809180
:1034D0004B048F5F80934B0492FE0AC08091670972
:1034E00082FD06C0772021F08FEF870D80934A047C
:1034F00093FE0BC08091670983FD07C080914A0449
:10350000833018F48F5F80934A041A82812C1982C9
:1035100050E2E52EF12C592D50725A87862D90E0FD
:103520009D878C87F5018491882309F42DC114911E
:1035300040904A0484100AC080914B0490E08215A8
:10354000930524F08FEF820D80934B0450904B0431
:10355000F981F51121C084101FC02A852223E1F0D2
:1035600000E028E048E0B7018E859F850E94D015D5
:103570001A3009F492C038F4173009F4ACC018308E
:1035800009F4B3C0C4C01D3009F4A0C0103279F0F2
:103590001B3009F0BCC0AEC01A3009F47EC008F47C
:1035A00098C01D3009F492C0103209F0A1C0C12C9E
:1035B000D12CF501EC0DFD1DE491E03221F43FEF3B
:1035C000C31AD30AF6CF49814C0D4F83C60143E09D
:1035D000880F991F4A95E1F799878887841043C01F
:1035E0009981591608F43FC0C601E9818E0F911DDB
:1035F000252D30E028173907B4F5871007C06E165F
:1036000028F02C853D852817390734F0C60195959B
:1036100087951981180F04C0561428F41981115088
:1036200010934B0405C0651418F43F8130934B048C
:103630004A85442371F000E028E04C2D440F440FEC
:10364000440FB7018E859F850E94D01550E25A83A2
:1036500014C048855985B7018E859F850E94123018
:1036600080E28A830AC028E04C2D440F440F440FA7
:10367000B7018E859F850E94902E91E0C91AD108CE
:10368000AC0CBD1CEF81E9832E853F8548855985AB
:10369000240F351F3F872E8773C0C50101960E94F6
:1036A00011161C018B819C8182199309880F991F27
:1036B000880F991FED81FE818E0F9F1F9F878E8738
:1036C000F8E0EF0EF11C839419825AC048E457E0E9
:1036D00004C0173041F446E357E0B7018E859F855B
:1036E0000E945E2C37C0183021F544E257E0F5CF38
:1036F0001B30F9F48091050190910601895F964095
:1037000019F449EE56E0E9CF49ED56E0E6CF8E8553
:103710009F8502969093860480938504C701019645
:10372000909384048093830461E0812F0E94351379
:1037300016C08E859F85029690938604809385049B
:10374000C7010196909384048093830460E0812FE5
:103750000E943513398135110AC0841008C048E031
:1037600050E0B7018E859F850E9412301A834E85E6
:103770005F85485F5F4F5F874E8759815F5F5983E1
:103780008FEFA81AB80ACECE95FC30C08091670999
:1037900085FF2CC09A819B3089F09D30E9F09730ED
:1037A000F9F48091050190910601805B964019F42F
:1037B00087E896E00CC080EB96E009C08091050197
:1037C00090910601895F964099F389EF96E0909376
:1037D0000601809305010AC08AE08093490403C072
:1037E0002A812093490489E00E9412179092670968
:1037F0003B85332309F444C020917B0430917C0441
:103800004091790450917A0410927C0410927B04C8
:1038100010927A041092790480917F049091800430
:10382000840F951F8A3191052CF0499790937A0463
:10383000809379048091810490918204820F931F78
:1038400097FD05C08937910534F088579109909309
:103850007C0480937B048091AF02882389F080915F
:10386000790490917A044817590739F480917B04C0
:1038700090917C042817390719F081E080931A0190
:103880002F960FB6F894DEBF0FBECDBFDF91CF915C
:103890001F910F91FF90EF90DF90CF90BF90AF906E
:1038A0009F908F907F906F905F904F903F902F9060
:1038B00008954F925F926F927F928F929F92AF92F4
:1038C000BF92CF92DF92EF92FF920F931F93CF930D
:1038D000DF936C013B012A010E9460118C01E3011E
:1038E000C017D1070CF046C0BE01C6010E9452119C
:1038F0008A3021F48E010F5F1F4F3CC08D30D1F311
:103900009E0126193709241535059CF5803261F191
:10391000C6010E9460115C014E017401EC1AFD0A9F
:103920008A149B0474F4B401C6010E9452118032BF
:1039300041F08A3031F08D3021F08FEF881A980AEB
:10394000ECCFEC0EFD1EC70186199709841595056D
:1039500014F4E701C5CFC615D70559F4C40DD51D1C
:103960008E010150110906C07E018FEFE81AF80A96
:10397000F0CF8E01C801DF91CF911F910F91FF9081
:10398000EF90DF90CF90BF90AF909F908F907F90FF
:103990006F905F904F90089540917304509174041C
:1039A000209171043091720442175307B4F490913E
:1039B000E8009570E1F39091E80092FD19C08093C2
:1039C000F100809173049091740401968F7399278C
:1039D000892B19F48EEF8093E80080917304909105
:1039E00074040196909374048093730481E00895A5
:1039F00080E00895DF92EF92FF920F931F93CF9391
:103A0000DF93D82E8A017B01E40EF51EEB01CE1563
:103A1000DF0571F0D7FE03C0FE01849101C08881EB
:103A20000E94CC1C21968111F2CF8FEF9FEF01C035
:103A3000C801DF91CF911F910F91FF90EF90DF9020
:103A400008952FB7F89487708093E9009091E8006B
:103A5000892F807295FF04C09091F20080E4891B49
:103A60002FBF0895615030F02091F100FC012083B8
:103A70000196F8CF289884E6809387040895CF9222
:103A8000DF92EF92FF920F931F93CF93DF936C011E
:103A90007A018B01C0E0D0E0CE15DF0581F0D801BE
:103AA0006D918D01D601ED91FC910190F081E02D99
:103AB000C6010995892B11F02196EECF7E01C70131
:103AC000DF91CF911F910F91FF90EF90DF90CF90FA
:103AD00008958091690481110DC082E0809365048E
:103AE00084E080936604109268041092670481E079
:103AF0008093690485E694E008950F931F93CF9314
:103B0000DF931F92CDB7DEB782E0898342E450E0B5
:103B100066ED77E080E80E94FA1C0E94691DDC01D6
:103B200012960D911C9113970115110589F0D8017A
:103B3000ED91FC910280F381E02DBE016F5F7F4F1C
:103B4000C801099597FD04C0F80100851185ECCFE7
:103B500089810F90DF91CF911F910F910895CF939D
:103B6000DF931F92CDB7DEB76983DC01ED91FC9145
:103B70000280F381E02D41E050E0BE016F5F7F4F96
:103B800009950F90DF91CF91089583E00E94211D48
:103B900090E00895FC018485958597FD0BC09FB743
:103BA000F89482E08093E9008091F2009FBF90E05A
:103BB000019608959FB7F89482E08093E900809180
:103BC000F2009FBF90E00895DC01FB0112968C91FA
:103BD000129790E02481358182179307D1F4918167
:103BE0008081813A31F481E0913091F0933089F411
:103BF00011C0813271F49B3021F482811F968C9325
:103C000005C09A3031F4828150968C9381E00895FA
:103C1000089580E00895DC01FB0188E4808389E455
:103C2000818384E482831D969C911D979F709F5B86
:103C300093831D968D919C911E9724E09695879570
:103C40002A95E1F78F708F5B848385E00895EF926A
:103C5000FF920F931F93CF93DF93FB0120812138B5
:103C600051F52381223239F5DC0112962C9130E096
:103C70004481558142175307F1F4EC010B851C85F3
:103C8000E12CF12C0115110591F0F80144815581C9
:103C90006281738180E80E94FA1C8F3FFFEF9F07CB
:103CA00069F0E80EF91ED8010D911C91EBCF81E06F
:103CB0008F87C70105C080E090E002C08FEF9FEFC3
:103CC000DF91CF911F910F91FF90EF900895CF93C7
:103CD000DF93CDB7DEB769970FB6F894DEBF0FBE9E
:103CE000CDBFFC01DB018C918F5F8C93BE016F5FB8
:103CF0007F4F89E1DB011D928A95E9F729E029834D
:103D000084E08A8391E09D8383E08E832A8721E289
:103D10002B879C879D879F8722E2288B27E02B8B10
:103D200025E02C8B8E8B20E430E0388F2F8B998F01
:103D300082818B8395858685998B8A8B8381806828
:103D40008D8B49E150E080E00E94FA1C69960FB625
:103D5000F894DEBF0FBECDBFDF91CF910895FC0177
:103D600082818F5BFB01808381E00895CF92DF9297
:103D7000EF92FF920F931F93CF93DF936C01EB01B0
:103D80007B01E40EF51E00E010E0CE15DF0581F0AA
:103D900069916D30D1F3D601ED91FC910190F081E4
:103DA000E02DC6010995892B19F00F5F1F4FEDCF4C
:103DB000C801DF91CF911F910F91FF90EF90DF909D
:103DC000CF9008950E94EA360C94B32A0F931F9364
:103DD000CF93DF931F92CDB7DEB78C01FC018485B2
:103DE000958597FF0EC0CE0101960E94492D01973F
:103DF00019F4898190E002C08FEF9FEFF801958759
:103E00008487F801848595850F90DF91CF911F916C
:103E10000F910895CF93DF931F92CDB7DEB7FC01CA
:103E20008485958597FD05C02FEF3FEF3587248763
:103E30000BC0CE0101960E94492D019719F489818A
:103E400090E002C08FEF9FEF0F90DF91CF91089528
:103E50001F920F920FB60F9211242F933F934F93FF
:103E60005F936F937F938F939F93AF93BF93CF9302
:103E7000EF93FF93C091E1008091E100837F8093F5
:103E8000E100C3FF0FC01092E90081E08093EB00D6
:103E90001092EC0082E38093ED001092880488E099
:103EA0008093F000C2FF18C00E94B32A809176046C
:103EB000882339F08091760481508093760488239A
:103EC00089F180918704882339F08091870481509B
:103ED00080938704882341F1C4FF10C08091E200E1
:103EE0008E7E81608093E2008091E1008F7E8093DE
:103EF000E1008091A5028E7E806111C0C0FF16C0D6
:103F00008091E2008E7E80618093E2008091E100EA
:103F10008E7E8093E1008091A5028E7E81608093E9
:103F2000A50204C05D9ACDCF289AD6CFFF91EF911C
:103F3000CF91BF91AF919F918F917F916F915F9141
:103F40004F913F912F910F900FBE0F901F9018959A
:103F50001F920F920FB60F921124CF92DF92EF9221
:103F6000FF920F931F932F933F934F935F936F9302
:103F70007F938F939F93AF93BF93EF93FF93CF93D1
:103F8000DF93CDB7DEB76C97DEBFCDBF1092E900EF
:103F90008091E80083FFFBC168E0CE0145960E9456
:103FA000321D82EF8093E8008D8987FF05C09091D4
:103FB000E80090FFFCCF03C09EEF9093E800982F9D
:103FC000907609F0C6C09E894F89588D2F89F88C4C
:103FD00091110CC0803829F48091A6028093F100E1
:103FE00002C01092F1001092F10045C1913051F4DD
:103FF000811141C14130510509F03DC18091A602B6
:104000008D7F0BC0933061F4811135C14130510572
:1040100009F031C18091A60282608093A6022BC173
:10402000953049F48091E80080FFFCCF822F8068B2
:104030008093E30020C1963009F05EC00B8D1C8D8B
:1040400022E01092E9001092740410927304F212AC
:1040500032C010927204109271040E947D1D99E08A
:10406000BE016F5F7F4FDB01E92F1D92EA95E9F7F3
:104070009983FA8291E09E8390EA98879AEF9987D4
:104080002091730430917404275F3F4F3C832B834E
:104090008D831092E90010927404109273041093AF
:1040A00072040093710449E050E080E00E94FA1C21
:1040B0000E947D1DE0C010937204009371040E9461
:1040C000691DDC0112960D911C91139701151105C4
:1040D00009F4BBC0D801ED91FC910480F581E02D7D
:1040E000BE016B5E7F4FC8010995009709F0C7C0FC
:1040F000F80100851185EACF973009F445C1983061
:1041000021F481E08093F100B6C0993009F0B3C08A
:10411000837009F039C1E8E0F1E081E031E096E335
:104120002081211109C08EE78093EA001092EA00F5
:104130008F89809388049FC08093E9003093EB00BF
:1041400021912093EC009093ED008F5F873041F731
:10415000EACF8B8D9C8D1092E9001092740410921E
:1041600073049093720480937104898D811153C0FC
:104170008E899D89913A49F4813209F005C147E061
:1041800050E062E171E080E0BBC0913209F0FCC018
:10419000833269F48F89988DA0E0B0E080930E019E
:1041A00090930F01A0931001B093110164C080326D
:1041B00069F48091E80082FFFCCF67E082E191E042
:1041C0000E94321D8BEF8093E80055C0823209F0C7
:1041D00052C08F8980931901EEEFFFE7859194918A
:1041E0008B3F9C4D19F0E0E0F8E002C0EEEFFAE002
:1041F0008091120190911301A0911401B0911501C9
:10420000803B9440A105B10509F09EC08091190141
:1042100080FF79C099C00E94691DFC010281138151
:104220000115110509F4B0C0D801ED91FC91019080
:10423000F081E02DBE016B5E7F4FC80109958111B1
:104240001AC0F80100851185EBCFF1E0FF1609F4E3
:104250004EC0F3E0FF1298C08F89882309F44AC04A
:10426000823089F440E867E08AE398E00E94613593
:10427000882309F489C08EEF8093E80088C018165F
:104280001906CCF381C0813029F440E86BE08EE25E
:1042900098E0ECCF833009F077C00E94691DDC0103
:1042A0001296ED90FC9013978E010F5F1F4F6801DF
:1042B000E114F10479F0D701ED91FC910680F781CA
:1042C000E02DB801C7010995080F111DF701E08421
:1042D000F184EECFD8011C92F60101900020E9F79D
:1042E0003197BF016C197D0940E0C601BFCF6CE179
:1042F00078E002C068E178E0FB01449150E080E89A
:104300000E94FA1CB8CFEE3F2AE0F20751F08081FC
:1043100091818737A7E79A0721F09093FF0A80934E
:10432000FE0A87E797E791838083809160008093FE
:1043300075049BE088E10FB6F894A895809360001F
:104340000FBE9093600097CF808191818737974708
:1043500009F091CFA89580916000886180936000FA
:104360008091750480936000EE3FBAE0FB0739F05E
:104370008091FE0A9091FF0A918380837CCF1092F6
:10438000FF0A1092FE0A77CF81E28093EB006C96D1
:104390000FB6F894DEBF0FBECDBFDF91CF91FF9176
:1043A000EF91BF91AF919F918F917F916F915F91AD
:1043B0004F913F912F911F910F91FF90EF90DF90C0
:1043C000CF900F900FBE0F901F9018957F928F92F5
:1043D0009F92AF92BF92CF92DF92EF92FF920F9394
:1043E0001F93CF93DF93C82E8B017A0180918804AD
:1043F000811103C08FEF9FEF74C08091A50280FFF1
:1044000005C08091E00082608093E000CE2DDF2D1A
:10441000D12C8AEFB82E8C2D8770982E8C2D80721F
:10442000882E8C2D8074782E9AE3A92E209719F46B
:10443000DD2009F451C08C2D0E94211D81110AC07C
:10444000BA94BB20B9F261E070E080E090E00E9495
:104450008C30ECCF282F30E0C217D3070CF48C2F10
:104460009FB7F8949092E9002091E80025FF32C0B0
:10447000282F30E0C21BD30B882029F08150A0F0F8
:104480001092F100FBCFF801C7FE0AC0815050F036
:1044900044914093F1003196F9CF41914093F1005E
:1044A0008150D8F7020F131FDD2019F0A092E80009
:1044B0000AC08091E80085FD08C0A092E800DD24D4
:1044C000D394209739F0D12C05C0209719F471109E
:1044D000A092E8009FBFAACF5D9884E680937604FF
:1044E000C701DF91CF911F910F91FF90EF90DF9067
:1044F000CF90BF90AF909F908F907F900895CF9373
:10450000DF93EC0180911901882331F083E00E9450
:10451000E6211816190634F081E090E09B838A8327
:1045200080E090E0DF91CF91089580915D0481114A
:104530006AC081E0809350048093510426E534E002
:104540003093530420935204109255041092540453
:1045500027E231E030934D0420934C04109258042C
:104560001092570410925A041092590480935B04DD
:1045700080935C0481EC809356040E94691DFC01C9
:1045800021818091500490E0820F911D0897C4F51D
:10459000A281B381109729F48CE494E09383828301
:1045A0000EC018968D919C911997009711F0DC011F
:1045B000F8CF8CE494E019969C938E9318978081A1
:1045C00080934E04818180934F04908180915104A7
:1045D000890F808380E090915004891788F4A0911E
:1045E0005204B0915304A80FB11D9C91A181B0E079
:1045F000A95FBE4F9C9391819F5F91838F5FEBCFAB
:1046000081E080935D048CE494E00895CF93DF9380
:10461000DC01683810F0685825C0E62FF0E067FF2D
:1046200012C0E058F10981E090E001C0880FEA95DE
:10463000EAF7809514969C911497892314968C938D
:10464000149760E00FC0EA5AF84F6491662321F195
:1046500067FF08C014968C9114978D7F14968C93E5
:1046600014976F77FD0186E0662321F09681691328
:1046700001C01682815031968111F6CFED010E9462
:104680009522AE014C5F5F4F28E030E062E00E946F
:10469000462F81E090E002C080E090E0DF91CF9172
:1046A0000895EF92FF921F93CF93DF93EC01162FA3
:1046B0000E946C237C01612FCE010E940623C7015A
:1046C0009927DF91CF911F91FF90EF900895089562
:1046D000089580E090E00895CF93DF93DC0168387F
:1046E00010F068582DC0E62FF0E067FF11C0E058C9
:1046F000F10981E090E001C0880FEA95EAF714968D
:104700009C911497892B14968C93149760E018C091
:10471000EA5AF84F6491611109C081E090E0139664
:104720009C938E93129780E090E046C067FF08C08C
:1047300014968C911497826014968C9314976F77CB
:1047400016968C911697681751F117968C911797BA
:10475000681729F118968C911897681701F1199626
:104760008C9119976817D9F01A968C911A97681737
:10477000B1F01B968C911B97681789F0FD01369656
:1047800080E090E02191211105C0FD01E80FF91FA3
:10479000668305C0019686309105A1F7BECFED0175
:1047A0000E949522AE014C5F5F4F28E030E062E04E
:1047B0000E94462F81E090E0DF91CF910895BC01E7
:1047C00080E090E00C948C308FB18095807F669B68
:1047D00088601C9B846008951F93CF93DF93EC0146
:1047E000162F0E946536181739F0612FCE01DF9120
:1047F000CF911F910C946D36DF91CF911F91089549
:1048000080389105B8F460347105A0F490E121E09E
:1048100061FD24E060FD220F62FD2295687F969F76
:10482000D0011124A80FA657BB4F8C91822B40FFBB
:1048300082278C93089580917D0490917E04009747
:1048400029F0936090937E0480937D0480917D0491
:1048500090917E0408953F924F925F926F927F9263
:104860008F929F92AF92BF92CF92DF92EF92FF9280
:104870000F931F93CF93DF9300D000D0CDB7DEB757
:1048800080916909853009F0BDC080916E0988303A
:1048900038F085E00E94471681E080931A01B2C08B
:1048A00020916C092983283008F094C0A0E12A9F48
:1048B000C00111248951974F9A838983DC018C911F
:1048C000882309F487C0109709F484C001E010E040
:1048D000E8E04E2E512C3D01BDE06B0E711CE980CD
:1048E000FA80ECE0EE0EF11CC980DA80FAE0CF0E1F
:1048F000D11CA980BA802FE0A20EB11C89809A80B9
:1049000088E0880E911CA981BA811E96BC83AB8376
:1049100080916E0990E0801791070CF473C0F2014A
:10492000E01BF10BD3018C91809FD001819FB00DD2
:104930001124CD0163E0959587956A95E1F79A83F7
:104940008983D7018C91809FA001819F500D1124F4
:1049500073E0559547957A95E1F7D6018D919C9135
:10496000089FB001099F700D189F700D1124D5018B
:104970002C912E9FC0012F9F900D1124680F791F3D
:1049800077FF02C0695F7F4F53E0759567955A9531
:10499000E1F7D4018D919C91089F9001099F300D02
:1049A000189F300D1124AB81BC813C903E9EC0010C
:1049B0003F9E900D1124820F931F97FD079629812A
:1049C00033E0959587953A95E1F70E94902E0F5F19
:1049D0001F4F9ECF85E00F900F900F900F90DF91AB
:1049E000CF911F910F91FF90EF90DF90CF90BF90EC
:1049F000AF909F908F907F906F905F904F903F907F
:104A00000C9447160F900F900F900F90DF91CF915D
:104A10001F910F91FF90EF90DF90CF90BF90AF90DC
:104A20009F908F907F906F905F904F903F900895F0
:104A300047EE58E020E030E08417950711F4822F0C
:104A400008952F5F3F4F405F5F4F28303105A1F73A
:104A50008FEF0895FC012081213039F10E94182543
:104A6000E7EAF2E020E030E091919F3F61F08917A2
:104A700031F02F5F3F4F28303105B1F704C02115C9
:104A8000310599F002C02FEF30E0D901A955BD4F93
:104A9000FD0192919C93DF01F2E0A73ABF07C1F7B5
:104AA0008093A70281E080931A010895CF93DF934A
:104AB000E7EEF8E020E030E0908191112EC0E901AE
:104AC00094E0CC0FDD1F9A95E1F7C951D74F888349
:104AD0007C836B831986188682E38C8782E390E05F
:104AE0009B878A875A834983E7EAF2E080E090E077
:104AF00041914F3F29F4FC01E955FD4F208304C04B
:104B0000019688309105A1F7CE010E942A2566E022
:104B1000CE010E946316CE0108C02F5F3F4F7096F2
:104B20002830310549F680E090E0DF91CF9108957B
:104B3000CF93DF93EC010E941825E7EAF2E020E032
:104B400030E091919F3FD1F0891731F02F5F3F4FB7
:104B500028303105B1F712C0F901E955FD4F8FEF4B
:104B60002730310519F48093AE0202C09181908301
:104B70002F5F3F4F31962830310591F7188281E041
:104B800080931A01DF91CF910895CF92DF92EF9237
:104B9000FF920F931F93CF93DF93EC0180916909EC
:104BA0008550823040F410916C09CE010E94182586
:104BB000181709F409C18091AF028823A1F08885F4
:104BC000998520917B0430917C04821B930B9987FB
:104BD00088878A859B852091790430917A04821B8D
:104BE000930B9B878A878881823009F4CEC010920C
:104BF0007E0410927D04833009F09EC06A857B8517
:104C000001E02D854C85888599850E94D0156A859F
:104C10007B852D854C85888599850E94902E8D8574
:104C20006A857B85680F711D888599854C850196FD
:104C30000E941E2B6A857B856F5F7F4F3C85888530
:104C4000998520E04D85830F911D0E94BE2A6A85BB
:104C50007B85685F7F4F4C85888599850E941E2BD8
:104C600002E010E04C8544506A857B85600F711F1F
:104C70008885998502960E941E2B0E5F1F4F083073
:104C8000110581F76E0125E0C20ED11CC6010E94FC
:104C90006011880F991F880F991F7C0197FF03C02F
:104CA0002FEFE21AF20AF594E794F194E194F108F7
:104CB00044E0480F6A857B856F5F7F4F2C85269582
:104CC00088859985820F911D8E0D9F1D01E026E03C
:104CD00002970E94D0154A855B854E5F5F4F8C8599
:104CE000869568857985680F711D6E0D7F1D20E0A2
:104CF000C6010E9418156A857B856F5F7F4F888586
:104D0000998527E047E004960E94D0156A857B8547
:104D10006E5F7F4F8885998525E045E005960E9466
:104D2000902E80916909823039F410916C09CE017E
:104D30000E9418251817F1F061E0CE010E94631659
:104D40008091AF02882309F43FC02885398580917E
:104D50007B0490917C04820F931F998788872A8512
:104D60003B858091790490917A04820F931F9B87F1
:104D70008A872AC06A857B856C5F7F4F8885998585
:104D800040E007960E940024D7CF6A857B8501E02A
:104D90002D854C85888599850E94D0156A857B85EF
:104DA0002D854C85888599850E94902E2D852450CF
:104DB0004C8544506A857B856E5F7F4F88859985D9
:104DC00002960E94902EB8CFDF91CF911F910F9144
:104DD000FF90EF90DF90CF9008952F923F924F92E7
:104DE0005F926F927F928F929F92AF92BF92CF927B
:104DF000DF92EF92FF920F931F93CF93DF93CDB784
:104E0000DEB728970FB6F894DEBF0FBECDBF5C01AA
:104E10002B018A01809189048F5F80938904FB01B3
:104E2000808191814817590710F451834083F5011F
:104E3000248580859185AC01420F511D5C834B8395
:104E40003A015AE0651A710822853385C90109962D
:104E50009E838D83E584F12CF901EE0DFF1DF8870B
:104E6000EF834701F9E28F1A9108690144E1C40E0A
:104E7000D11C0115110589F0F20140815181849EF8
:104E8000C001859E900D949E900D1124B8010E9442
:104E9000BC361B012C0C3D1C02C0212C312C8091F6
:104EA0006809823009F45AC058F4813009F01CC1F5
:104EB000FAE0EF1AF108C12CD12C442443941AC013
:104EC000833009F4F9C0843009F4BFC00DC1B401C6
:104ED000650D711D40E0C5010E940024542422E0AC
:104EE000A20EB11C4B815C814A155B0581F752E033
:104EF000C50ED11CCE14DF043CF45301512C8D801F
:104F00009E808C0C9D1CE3CF20E04E2D6D817E8118
:104F10008B819C810B970E94BE2A48E658E06D81E8
:104F20007E81C3010E945E2C6F8178856C5071096F
:104F300042E458E0C3010E945E2C012B09F4D4C066
:104F400001E029E049E0B101C3010E94D01529E048
:104F500049E0B101C3010E94902EC6C001151105A0
:104F600009F4C2C08091700990E0861597050CF491
:104F7000BBC0EB81FC818E179F070CF0B5C0809100
:104F8000720990E04D815E81841795070CF4ACC0E6
:104F90004F81588541505109841795070CF0A4C0E2
:104FA0002D5E3F4F2817390744F0F201808191812F
:104FB000009709F499C001970FC06F8178856B50F5
:104FC00071098617970774F0F2018081918180172B
:104FD000910708F089C001969183808381E08093D6
:104FE0001A017FC08215930594F0F8E02F0E311C52
:104FF0002816390664F0C5010E9420169A83898319
:10500000BE016F5F7F4F84E00E9453166AC0049711
:105010009601C816D9060CF49C01C4018C0D9D1D87
:10502000281739070CF4C9019C012C193D09209F50
:10503000C001219F900D309F900D1124B4010E945A
:10504000BC36F20171836083C9CF809169098430D5
:1050500009F04AC0C5010E9420169A838983BE01C7
:105060006F5F7F4F8CE699E00E942816882321F11C
:105070008091720990E004979601C816D9060CF445
:105080009C01C4018C0D9D1D281739070CF4C90122
:105090009C012C193D09209FC001219F900D309F3C
:1050A000900D1124B4010E94BC36F201718360831B
:1050B00081E080931A0118C0809169098430A1F4BD
:1050C000C5010E9420169A838983BE016F5F7F4FBE
:1050D0008CE699E00E942816882331F084E00E9433
:1050E00047168BE08093680928960FB6F894DEBFC8
:1050F0000FBECDBFDF91CF911F910F91FF90EF9029
:10510000DF90CF90BF90AF909F908F907F906F90E7
:105110005F904F903F902F9008952F923F924F9223
:105120005F926F927F928F929F92AF92BF92CF9237
:10513000DF92EF92FF920F931F93CF93DF93CDB740
:10514000DEB727970FB6F894DEBF0FBECDBFFC01C8
:105150002B831F830E83809189048F5F8093890442
:1051600080849184860E971EA284B384A40EB51EFB
:10517000022F10E004501109240122E0420E511CBC
:10518000F12C2C2C312CA1014E195F095D834C832D
:10519000AE81BF812C9130E02E193F09209FC001C4
:1051A000219F900D309F900D1124BA010E94D0369E
:1051B000640D751D3B01B4E06B1A7108650122E0B6
:1051C000C21AD10880916809823061F128F58130D6
:1051D00009F09CC001E025E04B81B501C4010E94AB
:1051E000D01525E04B81B501C4010E94902E4B8162
:1051F0004450B5016E5F7F4FC2010E941E2B28E014
:1052000048E0B601C3010E94D01528E048E0B6018D
:10521000C3010E94902E7AC0833009F45FC08430AD
:1052200041F174C02091700930E0261537050CF467
:105230006DC08091720990E08C159D050CF466C0DC
:105240006D5F7F4F621773070CF460C045E0A40EDA
:10525000B11CA816B9060CF459C0CF010E94201643
:105260009A838983BE016F5F7F4F87E00E94531648
:105270004AC080916909873009F048C0CF010E9477
:1052800020169A838983BE016F5F7F4F8CE699E079
:105290000E9428168823D1F12091700930E024194A
:1052A0003509AC81BD812A9FC0012B9F900D3A9F8B
:1052B000900D1124B8010E94D0366E0D7F1D6E1521
:1052C0007F052CF071016E157F050CF47B01EE81DA
:1052D000FF81E08281E080931A0118C08091690902
:1052E0008730A1F4CF010E9420169A838983BE01E2
:1052F0006F5F7F4F8CE699E00E942816882331F07B
:1053000087E00E9447168BE08093680927960FB6C6
:10531000F894DEBF0FBECDBFDF91CF911F910F91EB
:10532000FF90EF90DF90CF90BF90AF909F908F90C5
:105330007F906F905F904F903F902F900895AC01B9
:1053400080916809883089F4E0917704F0917804BD
:10535000309721F03C962591349102C020E030E056
:1053600081E06217730749F529C0209169093091DE
:105370006C09A7EAB2E09D919F3FD9F080E1989F28
:10538000F0011124E951F74F4E175F0759F480914E
:105390007D0490917E04682B792B70937E0460933A
:1053A0007D040BC08081823021F0253031F49313CD
:1053B00004C082E0AF3AB807F1F680E008952F927A
:1053C0003F924F925F926F927F928F929F92AF9295
:1053D000BF92CF92DF92EF92FF920F931F93CF93E2
:1053E000DF9300D000D000D0CDB7DEB74C017E8374
:1053F0006D832A01FC01808591855901A80EB91E93
:10540000828593857801E80EF91E809189048F5F6B
:1054100080938904CA010E946011880F991F880F28
:10542000991F3C01F2E06F0E711C650124E0C20E71
:10543000D11C930177FE02C02F5F3F4F3595279512
:10544000C21AD30A17014CE0240E311C8091700956
:1054500090E08A159B05A4F02091720930E02E158A
:105460003F0574F0A501485F5F4F4817590744F0A6
:10547000E1E0EC83A701455F5F4F421753070CF44F
:105480001C828C159D0594F02091720930E0221544
:10549000330564F0A3014C0D5D1D8417950734F4AA
:1054A00001E0C7014496281739070CF000E0C40159
:1054B0000E9420169A838983BE016F5F7F4F8AE620
:1054C00099E00E942816182FF0916809FB83F130AB
:1054D00019F0F230D1F02CC04D815E81B701C501C9
:1054E0000E945E2C0B81012728E0462DB101C601E8
:1054F0000E94D015A701435F5F4FB6016F5F7F4FDA
:10550000212FC2010E94181513C02C81211102C045
:10551000002371F0C4010E94201690936B098093C0
:105520006A098BE08093680981E080931A0101C0C9
:1055300010E0812F26960FB6F894DEBF0FBECDBFC8
:10554000DF91CF911F910F91FF90EF90DF90CF905F
:10555000BF90AF909F908F907F906F905F904F9093
:105560003F902F90089583E08093E9008091F200AE
:10557000882319F08AE38093E8000895DF92EF9280
:10558000FF920F931F93CF93DF937C01D22E8B0159
:10559000040F111DEB0177FF02C0C0E0D0E0C8018D
:1055A0000134110514F080E490E0C817D9073CF4E9
:1055B0004D2DBE01C7010E9400242196F0CFDF913E
:1055C000CF911F910F91FF90EF90DF9008959C0174
:1055D000240F311D1216130684F5803891056CF5E1
:1055E00097FF02C080E090E02138310514F020E8F8
:1055F00030E0281BFB01E770FF2741E050E001C0CD
:10560000440FEA95EAF7409577FF02C0695F7F4F44
:1056100033E0759567953A95E1F77695762F66278D
:1056200077956795860F971FFC01E657FB4F215032
:1056300020F0808184238193FACF0895603471052E
:1056400010F40C94E72A08957F928F929F92AF9264
:10565000BF92CF92DF92EF92FF920F931F93CF935F
:10566000DF9300D000D01F92CDB7DEB74C014B8343
:105670005C836D83909189049F5F90938904F4010A
:10568000808591856901C80ED91E82859385780130
:10569000E80EF91ECE0103960E946011880F991F33
:1056A000880F991F5C01F4E0AF0EB11C20917009C6
:1056B00030E02C153D059CF08091720990E08E152C
:1056C0009F056CF0A6014A0D5B1D241735073CF4BD
:1056D00011E09701265F3F4F821793070CF010E00F
:1056E00080916909813081F4C4010E9420169A8357
:1056F0008983BE016F5F7F4F8CE699E00E94281678
:10570000882319F0712E02C080E0712C0091680985
:10571000023009F440C0D0F5013009F062C007251D
:105720002AE04A2DB701C6010E94D015A7014E5F9D
:105730005F4FB6016E5F7F4F272DCE0103960E940B
:1057400018158EEF982E9A0C86010F5F1F4F492D6A
:10575000B701C8010E941E2BB701675F7F4F492D1B
:10576000C8010E941E2B2FEFE21AF20A20E048E047
:10577000B701C6010E94BE2AC6018A0D9B1D20E00A
:1057800048E0B70101970E94BE2A2BC00330E9F020
:105790000430A9F026C0112329F1C4010E9420166B
:1057A0009A838983BE016F5F7F4F81E00E94531609
:1057B00081E080931A018BE08093680912C08823EE
:1057C00081F081E080931A010CC0882351F081E0C0
:1057D0000E94471681E080931A018BE0809368094C
:1057E00001C010E0812F0F900F900F900F900F903D
:1057F000DF91CF911F910F91FF90EF90DF90CF90AD
:10580000BF90AF909F908F907F900895CF92DF923E
:10581000EF92FF920F931F93CF93DF9300D000D0AE
:105820001F92CDB7DEB77C01009789F460E080E37A
:105830000F900F900F900F900F90DF91CF911F91CD
:105840000F91FF90EF90DF90CF900C94351397FF5E
:1058500004C060E08DE20E943513CE0101966C0118
:10586000FC0100E010E02AE030E0C701B9010E942D
:10587000D036805D81937B010F5F1F4F053011058E
:1058800019F0E114F10489F70C0D1D1DC016D106A5
:1058900039F060E0F80182918F010E943513F6CF54
:1058A0000F900F900F900F900F90DF91CF911F915D
:1058B0000F91FF90EF90DF90CF9008958F929F927D
:1058C000AF92BF92CF92DF92EF92FF920F931F930E
:1058D000CF93DC019B014115510509F4B7C0FA01D2
:1058E000749131969491E72EF12C8D010E0D1F1DB0
:1058F000101611060CF0AAC0A038B1050CF0A6C015
:10590000F901E90FF11D1E161F060CF09FC020348F
:1059100031050CF09BC0C22FC770F90137FD3796D7
:1059200063E0F595E7956A95E1F78E2F37FF04C0A0
:10593000CC2311F08FEF8E0FB7FF05C0CC24DD24F0
:10594000CA1ADB0A02C0C12CD12C003811051CF088
:1059500020E82A1B01C0272F2C19082F082E000C25
:10596000110B8F3F1CF4602F609501C060E0F1E0E7
:10597000392F377009F4F0E0E92FE695E695E695C2
:10598000EF0F0E0F111D0930110514F0E8E0E81BB0
:10599000E61B382F360F10E83103A00DB11D11247E
:1059A000AC0DBD1DA657BB4FA22EB12C4E5F5F4F55
:1059B000769FC00CD11C1124CC0CDD1CCA018C0DAF
:1059C0009D1D00E810E00A191B09B7016A197B093F
:1059D000660F771F41E050E07A010C2E01C0EE0CFB
:1059E0000A94EAF75E2F822EFC019C2ECF93DF9360
:1059F000ED01EF96EF962296A590C590992059F06B
:105A0000AE9C5001CE9C600137302CF4F880D094CD
:105A1000FD20FB28F99233233AF0FC90C094FC203F
:105A2000FA28FD920C94152D11962A9529F75A956E
:105A300051F0282D33951124E60FF11DA00FB11D53
:105A4000C00FD11DD9CFDF91CF911124CF911F91DC
:105A50000F91FF90EF90DF90CF90BF90AF909F900D
:105A60008F900895DC01CB0160916809613081F469
:105A70001A96ED91FC911B97E20FF31F18966D910A
:105A80007C911997640F751F20E0AF010C941815D5
:105A9000089520918804211103C08FEF9FEF08958E
:105AA0005FB7F89422E02093E9002091F20030E003
:105AB0001216130614F421E030E0422FFC0184E6B4
:105AC000415038F02898809387049091F100919389
:105AD000F7CF2115310521F08091F200882319F0CC
:105AE0005FBFC90108958BE68093E800F9CF2F923C
:105AF0003F924F925F926F927F928F929F92AF925E
:105B0000BF92CF92DF92EF92FF920F931F93CF93AA
:105B1000DF9300D000D000D0CDB7DEB79E838D8359
:105B20004B013A01B02E26017093860460938504E0
:105B3000509384044093830426952695222E312C7D
:105B400087010E9460117C01C12CD12CCE14DF048E
:105B50006CF40115110551F0A101B6018D819E81F2
:105B60000E94591C6C0101501109F0CF8D819E815A
:105B70000E9460117C0193012B0D311D3C832B830E
:105B8000CE14DF040CF054C0A101B6018D819E81BA
:105B90000E94591C9A8389833601630189819A8105
:105BA0006816790654F5B3018D819E810E94C21159
:105BB000182F46145704C9F460918304709184042B
:105BC0008091850490918604AA2041F090938204EC
:105BD000809381047093800460937F0400E026E04A
:105BE00044E00E94D01561E001C060E0812F0E9476
:105BF00035133FEF631A730AD0CF6E147F040CF095
:105C0000BFCF80918304909184049C01295F3F4F12
:105C100030938404209383049092860480928504B8
:105C20000D962B813C81821793070CF4A9CF3AC0C3
:105C3000870101501109B8018D819E810E94C21116
:105C40008A3011F1B8018D819E810E94C2118D3080
:105C5000D9F04E145F0431F560918304709184048F
:105C60008091850490918604AA2041F0909382044B
:105C7000809381047093800460937F0400E026E0A9
:105C800044E00E94D0150EC080918304909184045A
:105C90000796909384048093830490928604809264
:105CA0008504D7CF26960FB6F894DEBF0FBECDBFC2
:105CB000DF91CF911F910F91FF90EF90DF90CF90E8
:105CC000BF90AF909F908F907F906F905F904F901C
:105CD0003F902F9008953FB7F8948091C20990911A
:105CE000C309A091C409B091C50926B5A89B05C0F8
:105CF0002F3F19F00196A11DB11D3FBFBA2FA92F4B
:105D0000982F8827820F911DA11DB11DBC01CD01C7
:105D100042E0660F771F881F991F4A95D1F70895B3
:105D2000EF92FF920F931F93CF93DF93EC018B01C0
:105D3000E42EF22E6034710510F40E94E72AB801B7
:105D40006F0D711D615071096034710520F44E2D85
:105D5000CE010E94E72A20E04F2DB801CE010E941B
:105D6000BE2ACE018E0D911D20E04F2DB801019766
:105D7000DF91CF911F910F91FF90EF900C94BE2A6D
:105D80002F923F924F925F926F927F928F929F924B
:105D9000AF92BF92CF92DF92EF92FF920F931F9339
:105DA000CF93DF93EC018B017A016901C61AD70A00
:105DB000D7FE03C0D194C194D10847018C1A9D0A23
:105DC00097FE03C09194819491088C149D0454F41F
:105DD0009E2D8F2D7901292F382F9C2F8D2FE80193
:105DE000092F182FEC16FD0654F4902F812F8901EE
:105DF000292F382F9C2F8D2FE701E92EF82E170120
:105E00002C1A3D0A2901401A510A57FE03C0519429
:105E100041945108310137FE03C08FEF681A780AA8
:105E2000759467940217130714F08FEF01C081E097
:105E3000A82E880FBB08EC16FD06ACF040E08C14D1
:105E40009D041CF4BE01C80102C0B801CE010E942D
:105E500000246418750877FE04C00A0D1B1D620C2F
:105E6000731C2196E8CFDF91CF911F910F91FF9086
:105E7000EF90DF90CF90BF90AF909F908F907F90EA
:105E80006F905F904F903F902F900895AF92BF9288
:105E9000CF92DF92EF92FF920F931F93CF93DF93F6
:105EA0001F92CDB7DEB77C0169836A01590141E0D9
:105EB00050E0BE016F5F7F4FFC0183810E94E621AD
:105EC0008C0197FD0BC0F7018381A501B6018064A9
:105ED0000E94E62197FD02C0800F911F0F90DF9175
:105EE000CF911F910F91FF90EF90DF90CF90BF90D7
:105EF000AF900895CF93DF9300D000D0CDB7DEB739
:105F00009091DA0899838A836B831C820E94952280
:105F100024E030E0AE014F5F5F4F61E00E94462F0A
:105F20000F900F900F900F90DF91CF910895CF9326
:105F3000DF93609172092091700930E0ADE7B9E01C
:105F400080E090E070E0FB01E80FF91FE034F1051C
:105F500018F543E0F595E7954A95E1F7F695FE2F9C
:105F6000EE27F795E795E20FF31FE657FB4F40E06A
:105F700050E0EA01C20FD31FC038D10520F4CC9104
:105F8000C083319611964F5F5F4F4830510589F7B6
:105F9000089688319105B9F6DF91CF910895ADE764
:105FA000B9E080E090E020917209FC01E20FF11D60
:105FB000E034F10574F08091C009811132C0609124
:105FC000720970E08091700943EF58E090E00C9402
:105FD0005E2C23E0F595E7952A95E1F7F695FE2FDF
:105FE000EE27F795E79520917009E20FF11DE6572E
:105FF000FB4F20E030E040917009B901640F711D42
:106000006038710524F440814C93319611962F5FCE
:106010003F4F2830310579F708968831910519F6F8
:10602000CACF08956F927F928F929F92AF92BF9244
:10603000CF92DF92EF92FF920F931F93CF93DF9354
:106040007C016B018A018091C6099091C709019674
:106050009093C7098093C60921E090E082FD20E07B
:10606000C22FD92F4E01C60107963C01570191E07E
:10607000A91AB108A00EB11E8016910694F440E052
:10608000B601C4018E0D9F1D0E94002440E0B301A3
:10609000C501881999090E94002482E0880E911C8C
:1060A000EBCF0E0D1F1D01501109BE016C0D7D1DA2
:1060B00040E0C8010E940024B3016C1B7D0B40E04E
:1060C000C7010E9400242296C830D10574F3DF91E5
:1060D000CF911F910F91FF90EF90DF90CF90BF90E5
:1060E000AF909F908F907F906F90089520919B0923
:1060F000282329F090919A09982381E009F080E003
:10610000089520919B09282329F490919A099823B6
:1061100081E009F480E008958F929F92AF92BF9240
:10612000CF92DF92EF92FF926B017C010E946B2E67
:106130004B015C01C114D104E104F104F1F00E94AF
:106140006B2EDC01CB0188199909AA09BB09883E8D
:106150009340A105B10570F321E0C21AD108E1080E
:10616000F10888EE880E83E0981EA11CB11CC114B2
:10617000D104E104F10419F7DDCFFF90EF90DF9037
:10618000CF90BF90AF909F908F9008951F920F92E5
:106190000FB60F9211242F933F938F939F93AF933A
:1061A000BF938091BC099091BD09A091BE09B091A7
:1061B000BF093091C10923E0230F2D3720F4019648
:1061C000A11DB11D05C026E8230F0296A11DB11D1A
:1061D0002093C1098093BC099093BD09A093BE0987
:1061E000B093BF098091C2099091C309A091C409DD
:1061F000B091C5090196A11DB11D8093C20990936C
:10620000C309A093C409B093C509BF91AF919F91F1
:106210008F913F912F910F900FBE0F901F90189567
:10622000CF93DF931F92CDB7DEB7789484B58260A9
:1062300084BD84B5816084BD85B5826085BD85B52A
:10624000816085BD80916E00816080936E001092A8
:106250008100809181008260809381008091810023
:1062600081608093810080918000816080938000B4
:106270008091910082608093910080919100816073
:106280008093910080919000816080939000809134
:10629000C10084608093C1008091C10082608093BE
:1062A000C1008091C10081608093C1008091C300D2
:1062B00081608093C3008091C00082608093C000A1
:1062C0008091C20081608093C20080917A008460D6
:1062D00080937A0080917A00826080937A00809126
:1062E0007A00816080937A0080917A008068809340
:1062F0007A00109288041092A6021092A502809152
:10630000D70081608093D70080EA8093D80089B558
:10631000806189BD89B5826089BD09B400FEFDCF69
:1063200061E070E080E090E00E948C308091D800C5
:106330008F7C80618093D8008091E000807F809383
:10634000E0008091E1008E7E8093E1008DE08093FB
:10635000E200559A209A81EC80937C0085B1806F91
:1063600085B984B1877E84B984B1876E84B95E9A19
:106370005F988AB1806D8AB9769A6E9881B3806F82
:1063800081BB899880B38D7080BB80E58CBD81E036
:106390008DBD85E090E00E94DF235F9A85E090E06C
:1063A0000E94DF235E985C98E0EAF2E08DEA92E0DA
:1063B00024912EBD00000DB407FEFDCF31968E173F
:1063C0009F07B1F75C9A81E8809364008091650033
:1063D0008160809365000E94E42387FF24C05C985D
:1063E00085EA8EBD00000DB407FEFDCF5C9A2E98A5
:1063F0002F982D988091640080628093640081E0E2
:1064000083BF889513BEFCCF2D980E94E423847827
:10641000843871F00E94E42384718431F9F088ECAF
:1064200090E00E94DF230E94E42382FDEDCF2CC088
:106430002D9A88EC90E00E94DF232F986FEF82E086
:1064400090E00E94EC2384EF91E00E94DF232F9ADA
:106450000E94E42384788438D9F3DCCF2D9A88EC29
:1064600090E00E94DF232E9860E082E090E00E949E
:10647000EC2384EF91E00E94DF232E9A0E94E42314
:1064800084718431D9F3CBCF2D9A80E180939C091C
:1064900083E884BD8FEF87BD81EF809380001092E9
:1064A000880010928A008FEF9FEF90939708809357
:1064B0009608E7EAF2E08FEA92E02FEF21938E1739
:1064C0009F07E1F780E48093700980E2809372096E
:1064D00040E050E06BE375E182E00E945625FC014C
:1064E0008AE090E0918780878EE090E093878287B2
:1064F0008CE6848784E285872FB7F8948091BC0965
:106500009091BD09A091BE09B091BF092FBF8093A2
:10651000B4029093B502A093B602B093B702EE24F2
:10652000E394F12CAAE8CA2EA4E0DA2EB6E0AB2E52
:10653000B5E0BB2E15E5212EE0E06E2EE0E07E2ECC
:106540008FB7F8944091BC095091BD096091BE0984
:106550007091BF098FBF8091B2029091B302840FF6
:10656000951F2091B4023091B502821B930B90933A
:10657000B3028093B2024093B4025093B502609389
:10658000B6027093B7028091B002882309F478C0F4
:1065900080E20E948130882329F068ED8BED98E03D
:1065A0000E946C2380E40E948130882329F067EDEB
:1065B0008BED98E00E946C2380E80E948130882354
:1065C00029F06AED8BED98E00E946C2380E10E9437
:1065D0008130882329F069ED8BED98E00E946C23CF
:1065E00088E00E948130882329F060E88BED98E0F4
:1065F0000E946C2384E00E948130882329F060EBA4
:106600008BED98E00E946C2380E20E947630882314
:1066100029F068ED8BED98E00E94062380E40E944B
:106620007630882329F067ED8BED98E00E940623F1
:1066300080E80E947630882329F06AED8BED98E09F
:106640000E94062380E10E947630882329F069EDBC
:106650008BED98E00E94062388E00E947630882324
:1066600029F060E88BED98E00E94062384E00E9408
:106670007630882329F060EB8BED98E00E940623AA
:106680008FB7F8944091BC095091BD096091BE0943
:106690007091BF098FBF80919D09242F281B822FE5
:1066A00090919E09992329F020939F0910929E09A9
:1066B000F9C190919C09291748F48F5F891708F058
:1066C000F1C181E083BF889513BEECC181E0809366
:1066D0009E0940939D09809198099091990901968E
:1066E00090939909809398098091B2029091B30296
:1066F00041970CF442C185E00E9412178091AF02CD
:1067000081112CC10E94972F0E94F215582E082F3C
:10671000017010E081FD05C022273327201B310BBB
:1067200003C09701201B310B52FA882480F8912C6A
:1067300053FC05C0882799278819990903C0C70108
:106740008819990921153105C9F0409173095091B3
:1067500074094115510531F43695322F22273795AA
:10676000279507C064E0220F331F6A95E1F7240FD5
:10677000351F309374092093730904C01092740973
:10678000109273090097C9F020917509309176092C
:106790002115310531F49695982F8827979587957F
:1067A00007C044E0880F991F4A95E1F7820F931FB5
:1067B000909376098093750904C01092760910921F
:1067C0007509409070093090720980917309909119
:1067D000740920916F093091700997FF0CC044270C
:1067E0005527481B590B2417350798F41092700948
:1067F00010926F0914C0009761F0AC01420F531F53
:106800004115504830F08FE78093700910926F095E
:1068100006C0820F931F9093700980936F09209197
:10682000750930917609809171099091720937FF4D
:106830000CC044275527421B530B8417950728F497
:10684000109272091092710910C0820F931F811566
:10685000A0E49A0730F0BFE3B09372091092710977
:1068600004C090937209809371098091700990E03F
:10687000841991099093790980937809209172097C
:1068800030E02319310930937B0920937A09409134
:10689000B002411139C04091C009552D5072598341
:1068A0004423C9F1009719F42115310579F040917D
:1068B0007C0950E0249FB001259F700D349F700D1E
:1068C0001124849F802D11240E947A2F80917709B2
:1068D0006981662359F085FD17C09091DA08892FE8
:1068E0008160981789F08093DA080AC085FF0CC090
:1068F0008091DA08982F9E7F80FF06C09093DA0877
:1069000060E080E00E947A2F5092770940927009EF
:106910003092720923C0892B11F4232B19F084E0E3
:106920000E941217809177099981992321F085FDA2
:1069300007C082E003C085FF03C083E00E941217F6
:106940005092770980917809480E409270098091A1
:106950007A09380E309272090E94CF2F80916E0909
:106960008F5F80936E098091B2029091B30240973D
:106970009093B3028093B202B7CE80911A01811135
:1069800021C08091B1028823D9F081E08093680909
:106990000E94972F8091A7028F3F41F0A0E18A9F2C
:1069A000C00111248951974F0E94C5258091AF02E3
:1069B000811102C00E94CF2F109268091092B1027B
:1069C00080E060C0109282041092810410928004D2
:1069D00010927F0481E0809368090E94972F84E5DC
:1069E00080938A04BAEAB0938B04EAE8F4E0228246
:1069F0002AEA23833296AE16BF06C9F784E5809350
:106A0000080588EA809309058AE095E09C012058F2
:106A10003F4FFC012E173F0729F020825AEA51838D
:106A20003296F8CFCF01AAE0B8E0AE17BF0771F7F2
:106A300085E18C938AE280930B0812968AE098E0B5
:106A400082589F4F2C922AEA11962C9311971296F6
:106A50008A179B07B9F725E5DC012C93E158FF4F16
:106A60008AE2808381E00E9412178091AF02811137
:106A700002C00E94CF2F1092680910921A01109242
:106A8000B10281E00E94C719F60180E0A0E0B8E001
:106A900000800EBC8111012C1197A0FDFDCF019249
:106AA000B9F70DB480919A0980939B090E94E42361
:106AB00080939A096114710409F442CD0E94000088
:106AC0003BCDDF92EF92FF920F931F93CF93DF9313
:106AD000D82EF92EE42E062F10E0C8010196880F5B
:106AE0000E94CC1C83E00E94CC1CCD2DDF2D0C0F0E
:106AF0001D1FC017D10789F0E7FE03C0FE01849176
:106B000001C088810E94CC1CF82E80E00E94CC1C21
:106B10008F2121968111EDCF01C081E0DF91CF91CE
:106B20001F910F91FF90EF90DF90089510928D08C4
:106B300010928C0888EE93E0A0E0B0E080938E087D
:106B400090938F08A0939008B093910883E391E00D
:106B500090938B0880938A088FEF9FEF909397080C
:106B6000809396081092DA088091A609811113C0CB
:106B70001092A1091092A0098EE898E09093A309C1
:106B80008093A20986E390E09093A5098093A409DD
:106B900081E08093A6090E949522FC01A385B4851B
:106BA000109729F480EA99E0948783870BC08D9130
:106BB0009C911197009711F0DC01F9CF80EA99E0E0
:106BC0008D939C93258536858091A4099091A50984
:106BD000820F931F968785871092DE081092DD083A
:106BE00085E491E09093DC088093DB088091B40900
:106BF000811113C01092AF091092AE0984EC98E095
:106C00009093B1098093B0098FE290E09093B3091B
:106C10008093B20981E08093B4090E949522FC011F
:106C2000A385B485109729F48EEA99E09487838729
:106C30000BC08D919C911197009711F0DC01F9CF59
:106C40008EEA99E08D939C93258536858091B209D3
:106C50009091B309820F931F96878587E7EEF8E03E
:106C6000168215821782709689E0E736F807C1F719
:106C70000E94F2158093670981E080937C098FEF71
:106C800080936A0980936B0980936C0980936D09E6
:106C900081E591E0909396098093950910929A0965
:106CA00010929B0980E180939C091092990910929F
:106CB000980910929E090895FC0105900020E9F7BB
:106CC000809590958E0F9F1F0895F999FECF92BDE4
:106CD00081BDF89A992780B50895262FF999FECF9E
:106CE0001FBA92BD81BD20BD0FB6F894FA9AF99AE9
:106CF0000FBE01960895052E97FB1EF400940E9486
:106D0000923657FD07D00E949A3607FC03D04EF406
:106D10000C94923650954095309521953F4F4F4FAA
:106D20005F4F089590958095709561957F4F8F4F37
:106D30009F4F0895A1E21A2EAA1BBB1BFD010DC097
:106D4000AA1FBB1FEE1FFF1FA217B307E407F5071B
:106D500020F0A21BB30BE40BF50B661F771F881FF7
:106D6000991F1A9469F760957095809590959B018D
:106D7000AC01BD01CF010895AA1BBB1B51E107C0A7
:106D8000AA1FBB1FA617B70710F0A61BB70B881FBB
:106D9000991F5A95A9F780959095BC01CD0108954A
:106DA00097FB072E16F4009407D077FD09D00E94B8
:106DB000BC3607FC05D03EF4909581959F4F089511
:106DC000709561957F4F0895EE0FFF1F0590F49128
:106DD000E02D099481E090E0F8940C94EF36F8945B
:026DE000FFCFE3
:106DE20001FFFFFFFF870600C18081000000FFFF57
:106DF200FFFF00E100000000000001C012802540FA
:106E020038004B00000000E41D671E271E0B1E0009
:106E1200000000AF1D7F22C51DE41ECA1D0A1FE629
:106E22001E000000005123B61E69236823000000E3
:046E320000672300D2
:00000001FF
